:100000000C94A9020C94D1020C94D1020C94D1024C
:100010000C94D1020C94D1020C946C030C94D10278
:100020000C94D1020C94D1020C94D1020C94D10204
:100030000C94D1020C94D1020C94D1020C94D102F4
:100040000C945F2B0C94D1020C94272F0C94672FE7
:100050000C94D1020C94D1020C94D1020C94D102D4
:100060000C94D1020C94D1020C94D1020C94D102C4
:100070000C94D1020C94D1020C94D1020C94D102B4
:100080000C94D1020C94D1020C94D1020C94D102A4
:100090000C94D1020C94D1020C94D1020C94D10294
:1000A0000C94D1020C94D1020C94D1020C94D10284
:1000B0000C94D1022D706C6561736520696E70754A
:1000C00074207363726970743A0072756E20736382
:1000D00072697074000D0A23000D0A23636F6D3A74
:1000E000000D0A23534E3A000D0A23444F43204883
:1000F000545450533A2F2F626A6C782E6F72672EC9
:10010000636E2F6E6F64652F3931340D0A23566587
:10011000723A50524F432D56312D323032313032F7
:1001200030312D346233346165390D0A236E616DCF
:10013000653A00736574207370656564206F6B2C7D
:1001400020000D0A73746F70206C656E28312C20AE
:1001500032293A20000D0A506172697479284E2CB8
:10016000204F2C2045293A200064617461206C6581
:100170006E28352D38293A2000706C656173652032
:10018000696E707574206E65772073706565643A6A
:10019000200063757272656E742073706565643AD1
:1001A0002000706C6561736520696E7075742067DE
:1001B0006174657761793A2000706C6561736520C0
:1001C000696E707574206E65746D61726B3A200093
:1001D000706C6561736520696E7075742069703A22
:1001E0002000746F646F2E2E2E0042796521000D61
:1001F0000A706C656173652073656C656374283182
:100200002D372C2071293A000D0A342E47455457BA
:1002100041593A20000D0A332E4E45544D41524B60
:100220003A20000D0A322E49503A20000D0A312E94
:10023000444843503A2000302E4D41433A20000DAF
:100240000A3D3D3D3D3D3D3D3D3D3D3D3D006F6BEE
:10025000212063616C6962726174696F6E3D006F29
:100260006B212063616C6962726174696F6E3D001D
:10027000292C2020507265737320746865202755DF
:1002800027206B657920616E6420686F6C642E2E68
:100290002E2E000D0A4F6E2074686520536572691A
:1002A000616C20636F6E736F6C6528002C20434176
:1002B0004C3233303430303D002C2043414C31310E
:1002C000353230303D002C2043414C35373630300C
:1002D0003D002C2043414C33383430303D006F73A7
:1002E000633D000D0A6572726F7200526574797019
:1002F00065206E6577207061737377643A20004ED5
:1003000065772070617373776F72643A2000427969
:1003100065210063757272656E7420706173737706
:100320006F72643A2000E2848300427965210052B2
:100330006573746F72652044656661756C742053D3
:10034000657420547275653F2100706C656173653A
:1003500020696E707574206E616D653A2000427977
:100360006521000D0A713A71756974006E3A63680F
:10037000616E6765206E616D653A003D3D3D736558
:10038000743D3D3D0D0A613A7265626F6F740D0AEE
:10039000623A726573746F72652064656661756C2C
:1003A00074207365740D0A633A6E6574776F726BAF
:1003B00020696E666F202620206D6F64690D0A64C7
:1003C0003A636F6D207365740D0A653A73657470D6
:1003D00061737377640D0A663A6D6F6469207363A5
:1003E0007269707420312D390D0A003D3D3D7363F3
:1003F0007269707420312D393D3D3D3D004F4646B8
:10040000004F4E00723A72657365742028333030A5
:100410006D73290D0A523A72657365742028352070
:10042000736563290D0A703A706F776572646F7730
:100430006E283330306D73290D0A503A706F77652E
:1004400072646F776E283520736563290D0A563AFA
:10045000566F75743D2000303A636F6D2073686588
:100460006C6C000D0A3D3D3D3D3D3D0069703D0019
:100470007061737377643A2000517569742E004679
:1004800061696C7572652E004F4B21000D0A235572
:100490007365204448435020746F20676574206959
:1004A000702C20706C6561736520776169742E2EE5
:1004B0002E00005EBCE2613FDD83C29C7E20A3FD76
:1004C0001F41009D23BE46DB65F88C11AF32CA5731
:1004D000E974090C0D080002010000030407000084
:1004E00000000000000000000000010204081020CD
:1004F00040800102040810200102040810200408B2
:1005000001020404040404040404020202020202BC
:100510000303030303030505050500000000230092
:10052000260029002C0000000000250028002B00D8
:100530002E0000000000240027002A002D00240EB9
:100540000B163D1B8D1F9B21322317252225792950
:10055000972F11241FBECFEFD8E0DEBFCDBF11E033
:10056000A0E0B1E0E2E1F7E702C005900D92A03A09
:10057000B107D9F724E0A0EAB1E001C01D92AB3089
:10058000B207E1F712E0C9EAD2E004C02197FE0108
:100590000E948D36CF39D107C9F70E94E8330C94F9
:1005A000873B0C9400000C94323B0C9486330C96E1
:1005B0000C94D3021F93CF93DF93EC01162F0E946C
:1005C000D702811741F0612FCE010C96DF91CF91B8
:1005D0001F910C943A3BDF91CF911F910895CF92D8
:1005E000DF92EF92FF921F93CF93DF93EC010E9473
:1005F000D702182FCE0101960E94D70290E0B0E0FA
:10060000A0E07C01DD24CC24F12ACE0102960E94D8
:10061000D702182FCE0103960E94D702C82AC7011D
:10062000B601712BDF91CF911F91FF90EF90DF907A
:10063000CF900895CF92DF92EF92FF92CF93DF9306
:10064000EC016A017B016F2D772788279927CE015E
:100650000E94DA02B70188279927CE0101960E94ED
:10066000DA0299278F2D7E2D6D2DCE0102960E94E4
:10067000DA026C2DCE010396DF91CF91FF90EF90BF
:10068000DF90CF900C94DA02611521EE720781059C
:100690009105F1F068F4611526E97207810591056D
:1006A00029F0613074488340910580F480E008951A
:1006B000611522EC720721E08207910559F061155E
:1006C00024E8720723E08207910559F783E0089533
:1006D00081E0089582E008951F920F920FB60F9265
:1006E00011242F933F934F935F936F937F938F9337
:1006F0009F93AF93BF93EF93FF93809121029091CB
:10070000220201969093220280932102809121027D
:100710009091220286309D4030F08091B401809308
:1007200066000C9400008091A5019091A6014E9660
:100730009093A6018093A5018091A5019091A601B7
:10074000893E934000F18091250290912602009706
:1007500029F001979093260280932502809123022D
:1007600090912402009729F001979093240280939E
:1007700023028091A5019091A601885E93409093F9
:10078000A6018093A5018091A3019091A401181660
:100790001906B4F48091A3019091A4014E9790930F
:1007A000A4018093A3018091A3019091A401181644
:1007B0001906A4F582E10E94B52D61E00197A1F52B
:1007C0008091A1019091A20118161906B4F48091AC
:1007D000A1019091A2014E979093A2018093A10153
:1007E0008091A1019091A201181619060CF583E1E0
:1007F0000E94B52D61E0019709F5FF91EF91BF913E
:10080000AF919F918F917F916F915F914F913F91A8
:100810002F910F900FBE0F901F90189582E10E94AC
:10082000B52D892B69F260E082E10E94872DC8CF47
:1008300083E10E94B52D892B01F360E083E10E94E2
:10084000872DDBCF9C018A309105B4F4982F9770E7
:100850002830310594F4906184B7877F84BF8091FC
:1008600060008861809360009093600080916000D8
:10087000806480936000089591E09062ECCFEF92E5
:10088000FF920F931F93CF93DF938BEB91E00E9426
:10089000942A6AEF70E080E090E00E94DA2B80E01A
:1008A00097EE9093360280933502E9ECF1E088E50B
:1008B000DF011D928A95E9F78F01C3E2D0E0CE01F6
:1008C0000E94D702F80181938F012196CB32D10586
:1008D000B1F711E0F8E01F9FE0011124C753DE4F8C
:1008E0007E0187E0E80EF11C1B3008F043C041E0B8
:1008F000BE018BEB91E00E94C42A8823D9F167E006
:10090000CE010E94482BD7019C918913EDCF909185
:10091000A0019F5F9093A00128819091C9012913A4
:1009200027C029819091CA01291322C02A81909160
:10093000CB0129131DC02B819091CC01291318C024
:100940002C819091CD01291313C02D819091CE015E
:1009500029130EC02E819091CF01291309C09091C7
:10096000D001891305C01092360210923502B2CF21
:100970001F5FB0CFDF91CF911F910F91FF90EF904C
:1009800008958BEB91E00E9480298BEB91E00E940F
:10099000902A41E064E48BEB91E00C94212ACF9201
:1009A000DF92EF92FF920F931F93CF93DF93CDB718
:1009B000DEB72C970FB6F894DEBF0FBECDBF082F61
:1009C00010E07801EE0CFF1CC7018B5C9D4F6C01A1
:1009D000FC018081918180349D4E1CF133E0000F39
:1009E000111F3A95E1F707531E4F8BEB91E00E94E0
:1009F0008029B8018BEB91E00E94712A40E06EEBF8
:100A00008BEB91E00E94212A68E0C8010E94482BEC
:100A1000F80190858917A1F080E097EEF6019183A7
:100A200080832C960FB6F894DEBF0FBECDBFDF914A
:100A3000CF911F910F91FF90EF90DF90CF9008958D
:100A40008E010F5F1F4F6E01FAE0CF0ED11C8BEBB2
:100A500091E00E94552AF80181938F01EC15FD0564
:100A6000B1F789819A8129812031A1F423E0880F8F
:100A7000991F2A95E1F72885203141F44F812CE018
:100A800030E0241B3109807F820F931FF701EB5C5C
:100A9000FD4FC5CF2D81207611F4887FF7CF20320E
:100AA00011F48C7FF3CF203489F78E7FEFCF0F9333
:100AB0001F93CF930E94C10460E273E080E090E056
:100AC0000E94DA2B09EC11E0C0E0F8018081882354
:100AD00019F08C2F0E94CF04CF5F085F1F4FCB30DF
:100AE000A1F7CF911F910F910895AF92BF92DF921E
:100AF000EF92FF920F931F93CF93DF9300D01F923B
:100B0000CDB7DEB72091A001222309F49AC09B83C0
:100B10008A8305E312E089ECE82E81E0F82ED12CDF
:100B2000D8018D919D918D0180349D4E0CF46EC045
:100B3000F7018081882309F471C0DD2059F0AA8172
:100B4000BB81ED91FC9111970190F081E02D6BE359
:100B5000CD010995AA81BB81ED91FC91119701907E
:100B6000F081E02D63E4CD0109958091A0018230F0
:100B700018F15701B5E0AB0EB11CE2E0E983D501F5
:100B80008D915D01803158F4AA81BB81ED91FC917A
:100B900011970190F081E02D60E3CD01099540E1CE
:100BA00050E0F501319760818A819B810E9472310A
:100BB000B981B13009F042C0AA81BB81ED91FC91AD
:100BC00011970190F081E02D6DE3CD010995F801B9
:100BD000329760817181072E000C880B990B0E945F
:100BE000113520E030E040E85DE30E94C635AB01FE
:100BF000BC0122E030E08A819B810E94873266E25C
:100C000073E08A819B810E946D30D394B8E0EB0E33
:100C1000F11CE2E00B341E0709F082CF8A819B8130
:100C20000F900F900F90DF91CF911F910F91FF9038
:100C3000EF90DF90BF90AF900C94A230F1E0F98379
:100C40009ECF0F900F900F90DF91CF911F910F913A
:100C5000FF90EF90DF90BF90AF900895CF92DF921A
:100C6000EF92FF920F931F93CF93DF93CDB7DEB731
:100C7000C954D1090FB6F894DEBF0FBECDBF9E0197
:100C80002F5F3F4F7901690110E000E0C8010E9429
:100C9000D702F60181936F010F5F1F4F09341105D1
:100CA000A9F78E818E3D39F48F818D3A21F48885A4
:100CB0008E3B09F4CDC08EED8E838DEA8F838EEB53
:100CC00088878091A001813071F48091D1018823BF
:100CD00051F0E1EDF1E0DE01949681918D9321E0F8
:100CE000E93DF207D1F767E0CE0184960E94482BD8
:100CF0009BA5891799F067E089EC91E00E94482B49
:100D00009091D0018913B4C0A9ECB1E0FE01B49672
:100D10008D91819331E0A13DB307D1F780E58DA797
:100D200082E58EA78FE48FA783E488AB89A58987A6
:100D30009AA59A872BA52B87422F022E000C550BC4
:100D40005F932F93292F092E000C330B3F939F9312
:100D5000282F082E000C330B3F938F938CE091E0EB
:100D60009F938F93CE01C1969F938F930E9491384A
:100D70008B8181500FB6F894DEBF0FBECDBF8E3F82
:100D800058F08091B4019FEF980F99839A8395E072
:100D9000980F9B838A508C832EE42C8740EC4D87E0
:100DA00038EA3E8791E09F8782E0888B8FEF898BBE
:100DB0008A8B8B8B1C8A4D8B3E8B9F8B988F198EC9
:100DC0009A8F92EC9B8F1C8E98E39D8F2E8F91E3D0
:100DD0009F8F18A219A21AA21BA224962FAF2497A4
:100DE00092E798AF96E799AF90E79AAF97E59BAFF8
:100DF00090E59CAF96E59DAF8EAF2A961FAE2A97E1
:100E000027961FAE279784E028968FAF289782ED0C
:100E100029968FAF299780E825968FAF25970BE409
:100E200010E060E0C8010E94DA020E5C1F4F0F3331
:100E3000F2E01F07B1F710E000E0F70161917F01D8
:100E4000C8010E94DA020F5F1F4F09341105A9F78C
:100E5000C75BDF4F0FB6F894DEBF0FBECDBFDF918B
:100E6000CF911F910F91FF90EF90DF90CF90089559
:100E7000188654CFFF920F931F93CF93DF938C016B
:100E8000EB0141E070E060E0CE010E942533F62ED8
:100E90004AE050E0CE010E947231E881F981019070
:100EA000F081E02D6EE2CE0109956F2DC8010E9400
:100EB000DA0241E070E060E0CE010E942533F62EB8
:100EC0004AE050E0CE010E947231E881F981019040
:100ED000F081E02D6EE2CE0109956F2DC8010196DB
:100EE0000E94DA0241E070E060E0CE010E9425330A
:100EF000F62E4AE050E0CE010E947231E881F9817D
:100F00000190F081E02D6EE2CE0109956F2DC801B0
:100F100002960E94DA0241E070E060E0CE010E9499
:100F20002533F62E4AE050E0CE010E9479316F2D34
:100F3000C8010396DF91CF911F910F91FF900C9400
:100F4000DA02CF93DF93EC0188E190E00E94EF0298
:100F5000AB01BC012AE030E0CE010E946531E8819E
:100F6000F9810190F081E02D6CE2CE01099588E2D3
:100F700090E00E94D302E881F9810190F081E02D98
:100F8000682FCE01099589E290E00E94D302E881A2
:100F9000F9810190F081E02D682FCE0109958AE258
:100FA00090E00E94D302E881F9810190F081E02D68
:100FB000682FCE01DF91CF910994CF9389E290E021
:100FC0000E94D3028E34C1F08F3409F457C08534A7
:100FD00021F58AE290E00E94D302C82F88E290E0D7
:100FE0000E94D302C133D1F5863309F478C070F57D
:100FF000853399F480E218C08AE290E00E94D3021F
:10100000C82F88E290E00E94D302C13379F486337E
:1010100009F461C020F4853331F086E005C08733E0
:10102000E1F784E001C080E0CF910895863309F4B0
:1010300054C020F4853389F788E0F6CF873321F058
:10104000883359F78EE0F0CF8CE0EECF873321F074
:10105000883319F786E2E8CF84E2E6CF863309F4D5
:1010600040C020F48533C9F688E2DECF873321F013
:10107000883399F68EE2D8CF8CE2D6CF8AE290E020
:101080000E94D302C82F88E290E00E94D302C133AD
:1010900089F4863341F128F4853309F0BECF80E32B
:1010A000C3CF873329F0883309F0B7CF86E3BCCFAD
:1010B00084E3BACF8633C9F028F4853309F0ADCF85
:1010C00088E3B2CF873329F0883309F0A6CF8EE3C7
:1010D000ABCF8CE3A9CF82E0A7CF8AE0A5CF82E295
:1010E000A3CF8AE2A1CF82E39FCF8AE39DCFCF93A4
:1010F000DF93EC016AE070E080E090E00E94DA2B80
:10110000E881F9810084F185E02DCE010995892BD4
:1011100041F0E881F9810284F385E02DCE01099543
:10112000EFCFDF91CF9108958F929F92AF92BF92B0
:10113000CF92DF92EF92FF92CF93DF93EC010E9468
:1011400077088FE190E00E94EF026B017C01C114EF
:10115000D104E104F104B9F063E173E0CE010E942F
:101160006D3041E070E060E0CE010E9425334B011C
:101170005C01CE010E94A2306EE073E0C814D90475
:10118000EA04FB0441F5CE010E9477086FEF72E09C
:10119000CE010E946D3041E070E060E0CE010E941F
:1011A00025336B017C01CE010E94A230CE010E944A
:1011B00077086BEE72E0CE010E946D3041E070E086
:1011C00060E0CE010E942533C616D706E806F90670
:1011D00079F063EE72E0CE01DF91CF91FF90EF9056
:1011E000DF90CF90BF90AF909F908F900C94A630DF
:1011F000CE010E94A230B701A6018FE190E0DF91FD
:10120000CF91FF90EF90DF90CF90BF90AF909F90E5
:101210008F900C941A03EF92FF920F931F93CF932A
:10122000DF931F92CDB7DEB707E212E0811102C053
:101230000BEA12E06FE372E0C8010E94A63067E398
:1012400072E0C8010E946D3085E0E82EF12CC701E4
:101250000E94D7028983803148F4D801ED91FC9136
:101260000190F081E02D60E3C801099540E150E074
:101270006981C8010E947231BFEFEB1AFB0A8BE053
:10128000E816F10421F76CE272E0C8010E946D30AB
:1012900087E190E00E94D3028983D801ED91FC910F
:1012A0000190F081E02D682FC801099589818F7D1B
:1012B0008E3409F072C063E272E0C8010E946D30A2
:1012C000F12CE12CC7010C960E94D70289834AE0D9
:1012D00050E0682FC8010E947231B3E0EB16F104B0
:1012E00049F0D801ED91FC910190F081E02D6EE282
:1012F000C8010995BFEFEB1AFB0A84E0E816F10478
:1013000009F765E172E0C8010E946D30F12CE12C13
:10131000C70140960E94D70289834AE050E0682FB7
:10132000C8010E947231A3E0EA16F10449F0D80125
:10133000ED91FC910190F081E02D6EE2C8010995DC
:10134000BFEFEB1AFB0A84E0E816F10409F768E046
:1013500072E0C8010E946D30F12CE12CC701449667
:101360000E94D70289834AE050E0682FC8010E949A
:101370007231A3E0EA16F10449F0D801ED91FC9135
:101380000190F081E02D6EE2C8010995BFEFEB1AE4
:10139000FB0A84E0E816F10409F76FEE71E0C8017A
:1013A0000E94A6301092220210922102C8010E94CF
:1013B000770841E050E0BE016F5F7F4FC8010E9497
:1013C0008633019769F06AEE71E0C8010E94A63089
:1013D0000F90DF91CF911F910F91FF90EF900895A3
:1013E00064E670E080E090E00E94DA2BD801ED9195
:1013F000FC910084F185E02DC8010995892B49F005
:10140000D801ED91FC910284F385E02DC801099586
:10141000EDCF8981823391F138F4803371F0F0F4AB
:101420008B3109F007CFD4CF8433E1F190F18135CE
:1014300079F2813709F0FECECBCF62EE71E0C801C0
:101440000E94A630C8010E94770841E050E0BE012A
:101450006F5F7F4FC8010E94D502ECCE87E190E01C
:101460000E94D3026EE4893509F069E58BE090E0D3
:101470000E94DA02C8010E947708DCCE60ED71E0BC
:10148000C8010E946D30B8018CE090E00E943A07DC
:10149000D1CE69EB71E0C8010E946D30B80180E1E6
:1014A00090E0F4CF62EA71E0C8010E946D30B801AB
:1014B00084E190E0EBCFCF92DF92EF92FF920F9317
:1014C0001F93CF93DF931F92CDB7DEB78C0162E9F4
:1014D00071E00E946D3088E190E00E94EF02AB0164
:1014E000BC012AE030E0C8010E94913169E771E057
:1014F000C8010E946D30C8010E9477084AE061E08F
:1015000070E0C8010E9425336A307105810591059C
:1015100008F495C0C12CB0E1DB2EBEE0EB2EF12C1F
:10152000613C27E2720729E08207910508F07AC042
:10153000C12CA8E0DA2EA7E0EA2EF12C613E23E9C7
:10154000720724E08207910508F06CC0C12CF4E812
:10155000DF2EF3E0EF2EF12C61322FEB720722E049
:101560008207910508F05EC0C12CE2ECDE2EEE246D
:10157000E394F12C613721E1720721E082079105A4
:1015800008F050C061382BEB72078105910508F017
:10159000D4C0613820E772078105910508F0D3C0F7
:1015A000C12C5BE4D52EE12CF12C613428E37207C9
:1015B00081059105B8F540E8C42E45E2D42EE12C12
:1015C000F12C61322CE172078105910558F530EC60
:1015D000C32E32E1D32EE12CF12C61312EE07207C3
:1015E00081059105F8F420E6C22E29E0D22EE12CE7
:1015F000F12C693027E072078105910598F4653870
:1016000023E072078105910508F0A3C0633C714097
:101610008105910508F0A4C08CE2C82EDD24D39486
:10162000E12CF12C2AE030E0B701A601C8010E94AC
:101630009131B701A60188E190E00E941A03C80128
:101640000E94770869E671E0C8010E946D3041E0B0
:1016500050E0BE016F5F7F4FC8010E948633019743
:1016600049F469818BEC860F843020F48CE190E0A2
:101670000E94DA0264E670E080E090E00E94DA2BDB
:10168000C8010E94770865E571E0C8010E946D30CD
:1016900041E050E0BE016F5F7F4FC8010E94D5025C
:1016A00089818F3611F48FE489838981853611F41D
:1016B00085E4898389818E3611F48EE4898369817A
:1016C000653421F082EB860F823020F48DE190E0CA
:1016D0000E94DA02C8010E94770862E471E0C80142
:1016E0000E946D3041E050E0BE016F5F7F4FC80146
:1016F0000E94D50269818FEC860F823020F48EE142
:1017000090E00E94DA0263E371E0C8010E946D304C
:10171000C8010E94A107C8010E94A230C8010E940E
:1017200077080E942E060F90DF91CF911F910F91A5
:10173000FF90EF90DF90CF900895C12C71EED72EDF
:10174000E12CF12C6FCFC12C66E9D62EE12CF12CC7
:1017500069CF90EBC92E94E0D92EE12CF12C62CF09
:1017600088E5C82E82E0D82EE12CF12C5BCF0F93B8
:101770001F93CF93DF938C01CCE2D0E0CE010E9487
:10178000D702882369F0D801ED91FC910190F08196
:10179000E02D682FC80109952196C733D10571F74F
:1017A000DF91CF911F910F910895FF920F931F9397
:1017B000CF93DF93EC0168EE70E00E946D30CE01B4
:1017C0000E94B70B61EE70E0CE010E946D3003E223
:1017D00010E0C8010E94D702F82E8FE08F1540F06C
:1017E000E881F9810190F081E02D60E3CE01099557
:1017F00040E150E06F2DCE010E9472310F5F1F4F0C
:101800000B32110531F769ED70E0CE010E946D30A9
:10181000CE010E94A10765ED70E0CE010E946D30FF
:10182000CE01DF91CF911F910F91FF900C94750520
:101830004F925F926F927F929F92AF92BF92CF92A0
:10184000DF92EF92FF920F931F93CF93DF937C0170
:101850006A018B015B012FEFA21AB20A0C151D055C
:1018600008F073C00E94A92B2B013C01A0E14A0E95
:10187000A7E25A1E611C711CD701ED91FC910084F6
:10188000F185E02DC7010995892B39F40E94A92B18
:10189000461657066806790678F70E94A92B461661
:1018A00057066806790608F450C0D701ED91FC91FF
:1018B0000284F385E02DC7010995EC01982ED7012C
:1018C000ED91FC910190F081E02D682FC701099501
:1018D000CE0199278A339105F4F4803391058CF475
:1018E0008D30910521F154F48830910511F10A975A
:1018F000F1F0992051F10F5F1F4FB0CF8D970297F4
:10190000C0F7692DC8010E94DA0260E0C8010196A3
:101910000E94DA02EECF8F35910599F32CF48154B1
:1019200091094A9730F7EDCF81569109FACF912C62
:10193000E8CFA016B106E8F6E801229760E0C801FA
:1019400001970E94DA028E01D4CFDF91CF911F91CF
:101950000F91FF90EF90DF90CF90BF90AF909F904E
:101960007F906F905F904F900895FF920F931F9319
:10197000CF93DF93EC01888199810E94D70210E018
:1019800000E09AE0F92E2881398190ED980F9A3085
:1019900080F4F09EA001F19E500D11248F708A01F9
:1019A000080F111DC9010196998388830E94D702EF
:1019B000EACF2150310939832883C801DF91CF91C3
:1019C0001F910F91FF90089501960E94D70290ED0C
:1019D000980F81E09A3008F080E00895CF92DF926E
:1019E000EF92FF920F931F93CF93DF9300D0CDB769
:1019F000DEB77C01162F22E3629FC0011124855BB4
:101A00009F4F9A8389836AEC70E0C7010E946D3012
:101A10004AE050E0612FC7010E94793189819A81A3
:101A20000E94D702182F18160CF0B4C011160CF033
:101A3000B1C0D701ED91FC910190F081E02D612FB3
:101A4000C7010995163509F43FC038F5123509F478
:101A50005FC0143509F481C0103521F5C980DA80E2
:101A6000C6010E94E40C882309F44AC0BFEFCB1AD8
:101A7000DB0ADA82C982CE0101960E94B50C9093EE
:101A8000A2018093A1016091A1017091A2014AE09D
:101A900050E0C7010E944C3105C01237C9F158F41B
:101AA0001037E1F289819A8101969A8389830E9495
:101AB000D702182FBBCF143709F44FC0163791F750
:101AC00060E083E00E94872DC980DA80C6010E9411
:101AD000E40C8823E1F18FEFC81AD80ADA82C982B0
:101AE000CE0101960E94B50C8C01BC0183E00E94DE
:101AF000712C4AE050E0B801C7010E948B31D2CF6F
:101B000061E0103509F060E083E10E94872DCACFC3
:101B1000C980DA80C6010E94E40C882391F02FEF7F
:101B2000C21AD20ADA82C982CE0101960E94B50C8D
:101B30009093A4018093A3016091A3017091A401EB
:101B4000A6CF61E0123509F060E082E1DECF61E00E
:101B5000163509F060E083E0D8CF09811A81C80109
:101B60000E94E40C882309F49DCF0F5F1F4F1A8356
:101B70000983CE0101960E94B50C8C014AE050E029
:101B8000BC01C7010E948B31B80190E080E00E9447
:101B9000DA2B88CF0F900F90DF91CF911F910F918B
:101BA000FF90EF90DF90CF900895CF92DF92EF9269
:101BB000FF920F931F93CF93DF937C01D62F0DE7F6
:101BC00010E0C1E0C8010E94D70298012E5C3F4F8F
:101BD0006901D11103C081508E3F48F54AE050E0C1
:101BE0006C2FC7010E947231D701ED91FC910190D9
:101BF000F081E02D6AE3C7010995C8010E94D70270
:101C00009FEF980F9E3F80F487FD09C0D701ED91AB
:101C1000FC910190F081E02D682FC70109950F5FBD
:101C20001F4FC016D10649F7C7010E94A230CF5FEF
:101C30008601CA3039F6DF91CF911F910F91FF9045
:101C4000EF90DF90CF9008950F9300E020E040E008
:101C500060E08BE492E00E94103087E292E00E9404
:101C6000A22061E18BEB91E00E94A12A67E170E084
:101C700085EB91E00E94012287EA91E00F910C949C
:101C8000A2200F931F93CF938C0164E670E080E055
:101C900090E00E94DA2BC8010E947708C8010E94D8
:101CA000A23061E0C8010E94D50DD801ED91FC91F0
:101CB0000084F185E02DC8010995892B29F4109243
:101CC000220210922102F1CFD801ED91FC91028401
:101CD000F385E02DC8010995C82F682F8BEA92E0A3
:101CE0000E947E2E2C2F2153330B29303105D8F43E
:101CF00064EB70E08BEA92E00E946D30CF708C2F25
:101D000090E0019622E3289FB001299F700D1124D5
:101D1000AB01455B5F4F675E7F4FC801CF911F915D
:101D20000F910C94180CCF911F910F910895CF92A1
:101D3000DF92EF92FF92CF938BEA92E00E945E2EA9
:101D40000E94A92B6B017C0120E1C20E27E2D21E6A
:101D5000E11CF11CC0E00E94A92B6C157D058E05CD
:101D60009F0580F5C730D8F10E94A92B6B017C013B
:101D700020E1C20E27E2D21EE11CF11CC0E00E944D
:101D8000A92B6C157D058E059F05F0F48BEA92E07A
:101D90000E94DE2D892B99F30E94A92B6B017C01F7
:101DA00020E1C20E27E2D21EE11CF11C8BEA92E078
:101DB0000E94FA2D8D3011F08A3069F5C73030F36A
:101DC00081E003C0C63080F680E0CF91FF90EF90B5
:101DD000DF90CF900895CF5F8B3209F0C0E08BEA9F
:101DE00092E00E94DE2D892B09F4B5CF0E94A92B29
:101DF0006B017C0120E1C20E27E2D21EE11CF11C26
:101E00008BEA92E00E94FA2D8D3011F08A3019F79A
:101E1000C73028F3A0CF982F9F7D953511F4CF5F61
:101E2000B5CF8B3209F4B2CFC0E0B0CF2F923F9242
:101E30004F925F926F927F928F929F92AF92BF92DA
:101E4000CF92DF92EF92FF920F931F93CF93DF9386
:101E5000CDB7DEB7C150D1400FB6F894DEBF0FBE8C
:101E6000CDBF982E809166009E012F5F3F4F790174
:101E700080E091E0D901FC011D923197E9F70BEA6E
:101E800012E0992011F007E212E088E190E00E9450
:101E9000EF022B013C016EED72E0C8010E946D3033
:101EA0004AE050E06091B401C8010E94723162EDD5
:101EB00072E0C8010E946D308CE090E00E94D30275
:101EC0004AE050E0682FC8010E94723166EC72E06F
:101ED000C8010E946D308DE090E00E94D3024AE07C
:101EE00050E0682FC8010E94723169EB72E0C801AE
:101EF0000E946D308EE090E00E94D3024AE050E0F4
:101F0000682FC8010E9472316CEA72E0C8010E9419
:101F10006D308FE090E00E94D3024AE050E0682FDD
:101F2000C8010E94793163E972E0C8010E946D30F6
:101F3000C8010E94A10760E772E0C8010E94A630B4
:101F4000D801ED91FC910680F781E02DC80109953B
:101F50000E94DD07282FB301A2018BEA92E00E94C4
:101F6000CB2E8BEA92E00E9477088BEA92E00E94E7
:101F7000DE2D0A97D4F38BEA92E00E94770800E006
:101F800011E080EB882E8091B401282F30E0E82DFD
:101F9000FF27E1950CF4F095E217F30714F0882E73
:101FA0008194C82C082C000CDD08A8014C195D098F
:101FB0004217530734F3880D809366008BEA92E052
:101FC0000E94770841E050E0BE016F5F7E4F8BEAD0
:101FD00092E00E94D502CF5FDE4F8881C150D14090
:101FE0008F7D8535D9F464E670E080E090E00E9452
:101FF000DA2B8BEA92E00E94770841E050E0BE01C4
:102000006F5F7E4F8BEA92E00E94D502CF5FDE4F7A
:102010008881C150D1408F7D853531F08394FFE4B4
:10202000F8150CF0B0CFADCF382CA12CBB24B39455
:10203000222423948091B401482F50E02FE42315EB
:102040000CF4B6C0032D032C000C110B9501201BC2
:10205000310B241735070CF4ABC0830D8093660059
:102060008BEA92E00E94770841E050E0BE016F5F8A
:102070007E4F8BEA92E00E94D502CF5FDE4F8881CF
:10208000C150D1408F7D853509F49EC064E670E073
:1020900080E090E00E94DA2B8BEA92E00E947708C1
:1020A00041E050E0BE016F5F7E4F8BEA92E00E94FC
:1020B000D502CF5FDE4F8881C150D1408F7D8535FD
:1020C00009F482C00C191D0917FF02C00F5F1F4FD2
:1020D00015950795080D8091B401800F80936600D7
:1020E0008090B401080DC301B2010E944403602F27
:1020F00090E00E94DA026FE572E08BEA92E00E94C3
:102100006D30609166004AE050E08BEA92E00E94F8
:102110007931992069F16EE472E087E292E00E94E1
:102120006D30609166004AE050E087E292E00E94E4
:1021300079314AE050E06091B40187E292E00E9478
:102140007231909166008091B401891798F56BE225
:1021500087E292E00E94AF1F609166008091B40117
:10216000681B770B4AE050E087E292E00E9453310F
:1021700068EE73E080E090E00E94DA2BCF5FDE4FE4
:102180000FB6F894DEBF0FBECDBFDF91CF911F9188
:102190000F91FF90EF90DF90CF90BF90AF909F9006
:1021A0008F907F906F905F904F903F902F90089509
:1021B000382C44CF6DE287E292E00E94AF1F8091FD
:1021C00066006091B401CCCF87E292E00E94C51F07
:1021D000882371F0609166004AE050E087E292E067
:1021E0000E947931E0916600EE0DFF2DF11D2082F5
:1021F000339420CFCF92DF92EF92FF920F931F93F1
:10220000CF93DF93CDB7DEB7AA970FB6F894DEBFB2
:102210000FBECDBF61E083E00E944B2D61E083E003
:102220000E94872D61E082E10E944B2D60E082E1F7
:102230000E94872D61E083E10E944B2D60E083E1E5
:102240000E94872D61E08DE00E944B2D61E08DE0C2
:102250000E94872D61E084E00E944B2D60E084E0C5
:102260000E94872D809166008093B4010E943F04F4
:1022700064E670E080E090E00E94DA2B0E9457054F
:1022800061E084E00E94872D8CE090E00E94D30200
:1022900081508E3F80F00E942E0626E040E052ECF6
:1022A00061E070E08BEA92E00E94CB2E8BEA92E034
:1022B0000E94160FE9CF0E942E0688E190E00E944E
:1022C000EF026B017C010E94440390E00E94D70260
:1022D00080936600C114D104E104F10431F4C12CEF
:1022E00082ECD82EEE24E394F12C0E94DD07282FF7
:1022F000B701A6018BEA92E00E94CB2E80E190E02C
:102300000E94D302682F83E00E94872D8EED8DA35B
:102310008DEA8EA38EEB8FA384E190E00E94D3021E
:1023200088A785E190E00E94D30289A786E190E02A
:102330000E94D3028AA78BE190E00E94D302082F6B
:102340008AE190E00E94D302F82E89E190E00E9499
:10235000D302182F88E190E00E94D3022F2D412F45
:10236000682FCE014F960E94103083E290E00E94C9
:10237000D302082F82E290E00E94D302F82E81E27D
:1023800090E00E94D302182F80E290E00E94D302D6
:102390002F2D412F682FCE0149960E9410308FE1DA
:1023A00090E00E94D302082F8EE190E00E94D302B9
:1023B000F82E8DE190E00E94D302182F8CE190E07E
:1023C0000E94D3022F2D412F682FCE0143960E94E9
:1023D00010308BEA92E00E94DE2D892B29F08BEAE7
:1023E00092E00E94FA2DF5CF87E190E00E94D3029F
:1023F0008E3409F44DC06CE874E08BEA92E00E94E0
:102400006D3016E08BEA92E00E94DE2D892B69F494
:102410006CE271E080E090E00E94DA2B6EE28BEAE1
:1024200092E00E947E2E115069F78BEA92E00E94A2
:10243000DE2D892B09F05DC0BE016B5D7F4F81E60B
:1024400092E00E94171E892BE9F068E874E08BEA9D
:1024500092E00E94A63085EB91E00E94BD2181E0D0
:1024600090E00E942204AA960FB6F894DEBF0FBE39
:10247000CDBFDF91CF911F910F91FF90EF90DF9033
:10248000CF9008956FE774E08BEA92E00E94A63047
:102490008FE891E09A8389834D895E896F89788D71
:1024A0004B835C836D837E8398878F834B8D5C8D9C
:1024B0006D8D7E8D49875A876B877C879E878D8738
:1024C00089A19AA1ABA1BCA18F87988BA98BBA8B4C
:1024D0008E010F5F1F4F9E01295F3F4FAE01435F8B
:1024E0005F4FBE016B5D7F4F81E692E00E94F51E5B
:1024F000B2CF69E774E0C8CF7F928F929F92AF927C
:10250000BF92CF92DF92EF92FF920F931F93CF93E0
:10251000DF93CDB7DEB7D2500FB6F894DEBF0FBE53
:10252000CDBF8BEA92E00E94770887E292E00E949A
:10253000770810E0109222021092210287E292E0C6
:102540000E94782181111AC087E292E00E9438210E
:1025500010923402DE5F0FB6F894DEBF0FBECDBF1F
:10256000DF91CF911F910F91FF90EF90DF90CF906F
:10257000BF90AF909F908F907F90089587E292E0F8
:102580000E94522018161906A4F487E292E00E94D5
:102590005D208D3009F448C08A3009F445C01F5FC2
:1025A0008B3209F010E0682F8BEA92E00E947E2EB9
:1025B000E5CF0E94A92B4B015C0120ED820E27E0A4
:1025C000921EA11CB11C8BEA92E00E94DE2D892B89
:1025D00009F4B0CFCE0101966C01F12CE12C782EDC
:1025E0000D2D8BEA92E00E94DE2D892B71F08BEA93
:1025F00092E00E94FA2DF60181936F01FFEFEF1A2E
:10260000FF0AE11422E0F20661F7A701672D702F9F
:1026100087E292E00E9436200E94A92B8616970638
:10262000A806B90680F686CF153008F4BBCF92CF46
:1026300087E292E00E94782181110C947C12089527
:102640004F925F926F927F92BF92CF92DF92EF9202
:10265000FF920F931F93CF93DF9300D000D000D051
:10266000CDB7DEB7B82E0BEA12E0882311F007E2EF
:1026700012E0C8010E94D50B40E25EE460E070E029
:10268000C8010E941F33BB2009F442C08FE190E0D3
:102690000E94EF026B017C01C114D104E104F1043A
:1026A000B9F160E774E0C8010E946D3041E070E06C
:1026B00060E0C8010E9425332B013C0187E292E0D3
:1026C0000E94C51F882321F087E292E00E947708CC
:1026D0008BEA92E00E947708C414D504E604F7045C
:1026E000B9F0C8010E94A23026960FB6F894DEBF5A
:1026F0000FBECDBFDF91CF911F910F91FF90EF9053
:10270000DF90CF90BF907F906F905F904F90089533
:102710006CE674E0C8010E946D3061E672E0CE01A3
:1027200001960E946A1FBE016F5F7F4FC8010E9421
:10273000983088E8E82E83E1F82E9CE2C92EDD244B
:10274000D394C8010E94770863E674E0C8010E9430
:10275000A630BB2029F067E574E0C8010E94A630CE
:1027600064E074E0C8010E946D3083E00E94B52DE2
:1027700061E074E0019711F06DEF73E0C8010E9411
:10278000A6306BEE73E0C8010E94A63060E0C8017D
:102790000E94D50D6BE773E0C8010E946D306CE6B6
:1027A00073E0C8010E946D30C8010E94B70B63E658
:1027B00073E0C8010E94A63041E050E0BE016F5FA7
:1027C0007F4FC8010E948633019731F06EE573E0B8
:1027D000C8010E94A63088CFC8010E94A230D8014B
:1027E000ED91FC910190F081E02D6981C80109957E
:1027F0006981E0EDE60FEB3408F0A3CFF0E0ED5F88
:10280000FB4E0C948D364E1454145414541454141A
:1028100054145414541454145414A113A113A11394
:10282000A113A113A113A113C514A81494149814EF
:102830009014A113A113A113A113A113A113A11308
:10284000A1135D14A1137814CC146E14A113A11359
:10285000A113A113A113A113A1139C14A113A113DC
:10286000A113A113A113A113C514A81494149814AF
:1028700090145914A113A113A113A113A113A1130F
:10288000A1135D14A1137314CC146914A113A11323
:10289000A1137D14A113A113A1139C14BB2009F44F
:1028A00050CF0E94181320CF6F70C8010E94EE0C09
:1028B00048CFC8010E94410E44CF6AE473E0C801CA
:1028C0000E946D3046E350E06CE270E0C8010E9467
:1028D000180CD092A401C092A30133CFF092A401AE
:1028E000E092A3012ECFD092A201C092A10129CFE4
:1028F000F092A201E092A10124CF83E00E94B52DC5
:1029000061E0892B09F060E083E00E94872D83E07D
:102910000E94B52D682F84E090E00E94DA0211CF6A
:10292000C8010E9494080DCF8B2D0E940B0909CF7E
:10293000C8010E945B0A05CF0E94A92B60347D402C
:102940008340910508F0FDCE8B2D0E94160FF9CE25
:102950006FE273E0C8010E94A63041E050E0BE0182
:102960006F5F7F4FC8010E948633019709F0E9CE5F
:1029700089818F7D893509F0E4CE60E086E090E0C2
:102980000E94DA020E942E06DCCE8091B401809370
:1029900066000C940000D5CE6AE273E0C8010E9484
:1029A000A630C8010E9477089FCECF93DF93CDB7A2
:1029B000DEB72D970FB6F894DEBF0FBECDBF1092D5
:1029C0002202109221028091250290912602892BE9
:1029D00041F48CE390E090932602809325020E94BC
:1029E000570565EB71E0CE0101960E94C1228B81F3
:1029F0009C819093AA018093A9018D819E81AF81D2
:102A0000B8858093AB019093AC01A093AD01B093D6
:102A1000AE0189859A85AB85BC858093AF01909383
:102A2000B001A093B101B093B2018D858093B30141
:102A300087EA91E00E94C51F882309F43FC067E23E
:102A400072E087EA91E00E94CD1F811137C080912A
:102A50003402882321F087E292E00E94382181E04D
:102A6000809334028091A9019091AA0190932A0247
:102A7000809329028091AB019091AC01A091AD01AE
:102A8000B091AE0180932B0290932C02A0932D0263
:102A9000B0932E028091AF019091B001A091B1014D
:102AA000B091B20180932F0290933002A093310233
:102AB000B09332028091B30180933302809134024B
:102AC000882301F187E292E00E94782181110FC0F2
:102AD00087E292E00E943821109234022D960FB6C0
:102AE000F894DEBF0FBECDBFDF91CF91089587E28E
:102AF00092E00E9452201816190684F781E00E9485
:102B00002013ECCF0E94970E882341F380E0F7CF8B
:102B1000CF93CFB7F89480915402811127C0ECE095
:102B2000F5E08491E4EFF4E09491E82FF0E0EE0F0B
:102B3000FF1FEE5CFA4FA591B491EC91E92321F4CB
:102B400061E08AE00E94872D61E08AE00E944B2DBF
:102B50008CB580618CBD8CB580648CBD61E08DE0EE
:102B60000E944B2D61E08BE00E944B2D809154021E
:102B70008F5F80935402CFBFCF9108950E9624E1CA
:102B8000FC0111922A95E9F70895CF93DF93EC01A8
:102B9000625F7F4F0E941C30CE01DF91CF9108957C
:102BA000CF93DF93EC016A5E7F4F0E941C30CE0111
:102BB000DF91CF910895CF93DF93EC01665E7F4F55
:102BC0000E941C30CE01DF91CF910895CF93DF9307
:102BD000EC016E5D7F4F0E941C30CE01DF91CF91E2
:102BE0000895FC01828993890895FC01848995895F
:102BF000089580E3FB0180833296842F82958F7045
:102C00004F704A3030F4405D4293482F8111F5CF28
:102C10000895495CF9CF0F9300E020E040E060E0C8
:102C200085E592E00E9410300F9108957F928F9277
:102C30009F92AF92BF92CF92DF92EF92FF920F934B
:102C40001F93CF93DF93CDB7DEB7AC970FB6F89451
:102C5000DEBF0FBECDBF7C01762E942E852E20E2E6
:102C6000A22ECE0101966C01DC01EA2D1D92EA959F
:102C7000E9F70FEF2FEF4FEF6FEF86960E941030BE
:102C80008701055B1F4F8FE891E09AA389A389A56F
:102C90009AA5ABA5BCA58BA39CA3ADA3BEA343E4FF
:102CA00050E0BE016F5D7F4FC8010E949B230196DB
:102CB00009F4C5C081E089838A8386E0B82EBB828F
:102CC0001C82D70114966D917D918D919C911797DF
:102CD0000E9493366D837E838F83988789869A8638
:102CE00080E890E09C878B874CE150E0B601C801FA
:102CF0000E94A723FE0137968AE1DF011D928A9583
:102D0000E9F74701B8E08B0E911CF401D601019060
:102D10000D92BA94E1F740E150E0B601C8010E947B
:102D2000A723F6011192AA94E9F796E0A92EB12CF7
:102D300040E250E0B601C8010E94A723F1E0AF1ABB
:102D4000B108B1F783E6898392E89A8393E59B8380
:102D50008C8385E38D8381E08E837F829DE39887DA
:102D600097E099878A8786E0F401DE011B9601903F
:102D70000D928A95E1F78CE0898B8A8B6AE171E08C
:102D8000CE0143960E948A38D7011B964C91BE0112
:102D9000675E7F4FC7010E94F915F7014485BE01A8
:102DA000655E7F4FC7010E94F915D7011D964C91B2
:102DB000BE01635E7F4FC7010E94F9154EE150E0EE
:102DC000B601C8010E94A723B3E07B121EC082E3B4
:102DD000898384E08A83F70196859B8397859C830A
:102DE00090899D8391899E8396E39F838887868DB2
:102DF0008987878D8A8780A18B8781A18C874CE00A
:102E000050E0B601C8010E94A72387E3898386E0CA
:102E10008A8391E09B8393E09C838D838FE08E83F4
:102E20008AE38F838BE388878FEF898749E050E0BF
:102E3000B601C8010E94A723C8010E94A323AC9633
:102E40000FB6F894DEBF0FBECDBFDF91CF911F91BB
:102E50000F91FF90EF90DF90CF90BF90AF909F9039
:102E60008F907F9008952F923F924F925F926F9232
:102E70007F928F929F92AF92BF92DF92EF92FF92DA
:102E80000F931F93CF93DF93CDB7DEB7E4970FB6C1
:102E9000F894DEBF0FBECDBF7C014A015B01190172
:102EA0000E94A92B2B013C018701055B1F4FC80124
:102EB0000E941C24181619069CF00E94A92B641964
:102EC00075098609970986169706A806B90608F4B3
:102ED000C6C162E370E080E090E00E94DA2BE7CFA9
:102EE00042E250E0BE016F5F7F4FC8010E94E523C0
:102EF0008981823009F0AEC1F801858996898334D1
:102F0000910509F0A7C16D817E818F8198850E940E
:102F100093362B013C01F10140825182628273821F
:102F200046E050E0B701685F7F4FCE014D960E94AA
:102F30007D38892B99F4F70180819181A281B38139
:102F4000481659066A067B0648F084819581A68159
:102F5000B78184159505A605B705E8F4C8010E9458
:102F60007423D12C8D2DE4960FB6F894DEBF0FBEDE
:102F7000CDBFDF91CF911F910F91FF90EF90DF9028
:102F8000BF90AF909F908F907F906F905F904F9089
:102F90003F902F90089589899A89AB89BC8986874B
:102FA0009787A08BB18B8EECA82EB12CC8010E9404
:102FB000BB23F1E0AF1AB108C9F7D12CC7014E9677
:102FC0004C01F701E45AFF4FFAA7E9A740969CA7E6
:102FD0008BA7F297FEA7EDA7089798AB8FA77097DE
:102FE000FAABE9AB1701F2E22F0E311C40979CAB14
:102FF0008BABC8010E945A23181619060CF02BC17E
:10300000C8010E94BB238F30910509F4A8C08CF53C
:103010008330910509F46CC08CF4009751F301974B
:1030200009F45BC0C8010E94BB23B82EBA94FFEF1D
:10303000BF16F9F2C8010E94BB23F8CF8630910574
:1030400009F472C00C9771F7C8010E94BB235C01A0
:10305000BB24C50101960E94B436F701958B848B81
:10306000A501BC01C8010E94E523F7018489958967
:103070008AC08633910509F48BC074F483339105BB
:1030800009F4CEC0C59771F6C8010E94BB23C801E0
:103090000E94BB23D82EADCF8B33910509F4AAC073
:1030A0008F3F910509F4A5CFCA9709F0BBCFC8019E
:1030B0000E94BB2344E050E06DA57EA5C8010E949C
:1030C000E523F70162A573A584A595A50E94933613
:1030D00062A773A784A795A78CCFC8010E94BB23C2
:1030E00044E050E06BA97CA9C8010E94E52381CF90
:1030F000C8010E94BB23A82E44E050E069A97AA928
:10310000C8010E94E523712C612CEA2DE450FF0BCD
:103110005F016A147B040CF06CCFC8010E94BB23D2
:10312000FFEF6F1A7F0AF5CFC8010E94BB23A82EBC
:1031300044E050E0B101C8010E94E523712C612CEC
:103140008A2D8450990B5C016A147B040CF051CFDA
:10315000C8010E94BB239FEF691A790AF5CFC80105
:103160000E94BB235C01BB24C50101960E94B436BA
:10317000F701938B828BA501BC01C8010E94E52356
:10318000F70182899389A80EB91EF501108231CF0B
:10319000C8010E94BB23B82EF701868D811109C09A
:1031A000878D811106C080A1811103C081A1882370
:1031B000A1F0E9A5FAA54080518062807380B40136
:1031C000CE0183960E941C308DA19EA1AFA1B8A50F
:1031D00084159505A605B70521F444E050E0B40137
:1031E00083CFBA94FFEFBF1609F403CFC8010E9442
:1031F000BB23F7CFC8010E94BB2344E050E06BA57E
:103200007CA5C8010E94E523F70166A577A580A9E2
:1032100091A90E94933666A777A780AB91ABE9CEC0
:10322000C8010E94BB2344E050E06FA578A9C80103
:103230000E94E523F70166A177A180A591A50E94D0
:10324000933666A377A380A791A762AB73AB84ABD9
:1032500095ABCFCED12CC8010E94742383CEDD2440
:10326000DA9480CE2F923F924F925F926F927F922C
:103270008F929F92AF92BF92CF92DF92EF92FF9286
:103280000F931F93CF93DF93CDB7DEB729970FB678
:10329000F894DEBF0FBECDBF8C0120ED37E040E0DB
:1032A00050E061E070E080E090E00E94C933D80116
:1032B00014966D937D938D939C931797F80160837B
:1032C0007183828393835801FBE4AF0EB11CC50167
:1032D0000E94862364E470E0C5010E946F24882365
:1032E00009F438C10E94A92B2B013C0148018AE452
:1032F000880E911C180192E4290E311C48EEC42E50
:1033000043E0D42EE12CF12CD801DE96B987A887B2
:103310001F821E82F40180818330A9F181115DC07A
:10332000F80184819581A681B7810196A11DB11D07
:1033300084839583A683B7830E94A92B641975099A
:1033400086099709A70196010E944C36A90161E000
:10335000C8010E94161681E0D4018C938E819F8152
:103360000197C1F20E94A92B641975098609970972
:10337000A885B9852D913D914D915C912617370710
:103380004807590728F6C5010E948623F801848161
:103390009581A681B7810196A11DB11D8483958376
:1033A000A683B7838E819F8129960FB6F894DEBFDE
:1033B0000FBECDBFDF91CF911F910F91FF90EF9086
:1033C000DF90CF90BF90AF909F908F907F906F9045
:1033D0005F904F903F902F9008958430F9F4F8015A
:1033E00084819581A681B7810196A11DB11D848339
:1033F0009583A683B7830E94A92B64197509860952
:103400009709A70196010E944C36A90163E0C80103
:103410000E941616E2E0D401EC93A0CF813049F56A
:10342000D1014D915D916D917C919E012F5F3F4F38
:10343000C8010E9433178D83823009F084C08981CE
:103440009A81AB81BC81F80184839583A683B7837D
:103450000E94A92B6419750986099709A70196018D
:103460000E944C36A90163E0C8010E941616ED8146
:10347000D2CF823009F072CFD1014D915D916D9123
:103480007C919E012F5F3F4FC8010E9433178D83AF
:10349000853009F052C083E0F4018083F80186A1F1
:1034A00097A1A0A5B1A5892B8A2B8B2B41F484E889
:1034B00093E0A0E0B0E086A397A3A0A7B1A7F8018E
:1034C00082A593A5A4A5B5A5892B8A2B8B2B61F486
:1034D00086A197A1A0A5B1A5B695A7959795879523
:1034E00082A793A7A4A7B5A7F80182A593A5A4A531
:1034F000B5A546A557A560A971A9452B462B472B15
:1035000051F4AC01BD01440F551F661F771F46A73C
:1035100057A760AB71ABF80182AB93ABA4ABB5AB73
:1035200086A597A5A0A9B1A986AB97ABA0AFB1AF6F
:1035300081E090E09F838E8311CF9D81963019F4B6
:10354000D4011C920BCFBD81BF3F09F007CFF4011E
:10355000108204CF1F821E8225CFCF92DF92EF927E
:10356000FF920F931F93CF93DF93EC016B011EA289
:103570001FA218A619A61AA61BA61CA61DA61EA643
:103580001FA618AA19AA1AAE1BAE1CAE1DAEFC01CE
:10359000FE9620833183428353833496E082F18206
:1035A000028313838C01085F1F4F86E0F80111929C
:1035B0008A95E9F7CE010E94BE1586E0F601D80192
:1035C00001900D928A95E1F7FE01E65BFF4F1082B4
:1035D000CE01DF91CF911F910F91FF90EF90DF907F
:1035E000CF900C943219FB01428153816481758123
:1035F000FC01428353836483758317821682089586
:10360000FB01DB018D918111FDCF90E080E070E046
:1036100060E03AE021912223F9F06430710554F51D
:103620002E3271F48F3F910509F024F5DA01A60FCF
:10363000B71F12968C936F5F7F4F90E080E0EACFC8
:10364000389FD001399FB00D1124822F220F990B82
:10365000C0978A0F9B1FDECF8F3F910509F054F46E
:10366000643071053CF4460F571FFA01828381E0F4
:1036700090E0089590E080E008950F9300E020E04E
:1036800040E060E08BE592E00E9410300F910895D9
:103690008F929F92AF92BF92CF92DF92EF92FF9262
:1036A0000F931F93CF93DF9300D01F92CDB7DEB758
:1036B0006C017B010E94A92BF6017783668386014A
:1036C000085F1F4FB6016A5F7F4F42E050E0C801BC
:1036D0000E94A72381E090E09A83898342E050E032
:1036E000BE016F5F7F4FC8010E94A72380E091E079
:1036F0009A83898342E050E0BE016F5F7F4FC8012B
:103700000E94A7231A82198242E050E0BE016F5F37
:103710007F4FC8010E94A72342E050E0BE016F5FC7
:103720007F4FC8010E94A72342E050E0BE016F5FB7
:103730007F4FC8010E94A7236701F701808188237A
:1037400001F17601F70181915F01882311F08E323A
:10375000B1F447018C189D081814190474F48B8275
:1037600041E050E0BE016D5F7F4FC8010E94A7237A
:10377000A401B601C8010E94A7236501DECF75012F
:10378000E1CF1B8241E050E0BE016D5F7F4FC80179
:103790000E94A723E12CFF24F394FA82E98242E0FD
:1037A00050E0BE016F5F7F4FC8010E94A723FA82DD
:1037B000E98242E050E0BE016F5F7F4FC8010E9486
:1037C000A72381E090E00F900F900F90DF91CF91B1
:1037D0001F910F91FF90EF90DF90CF90BF90AF902F
:1037E0009F908F9008952F923F924F925F926F9289
:1037F0007F928F929F92AF92BF92CF92DF92EF9281
:10380000FF920F931F93CF93DF93CDB7DEB76397EC
:103810000FB6F894DEBF0FBECDBF7C012B011A019D
:103820000E94A92B4B015C018701085F1F4F712C7F
:10383000612CC8010E941C24181619069CF00E94D5
:10384000A92B681979098A099B0946165706680643
:10385000790608F431C162E370E080E090E00E94F4
:10386000DA2BE7CFF7014281538164817581818D25
:10387000928DA38DB48D481759076A077B0709F00D
:103880001FC1858D968DC59709F01AC1C8010E9488
:103890005A230C970CF419C14CE050E0BE016F5F45
:1038A0007F4FC8010E94E5238B819C81982789273F
:1038B00098279A8B898BF7014681578129813A8114
:1038C0004217530711F497FD21C0C8010E947423C9
:1038D0007CEFE72EFF24FA94C70163960FB6F894A5
:1038E000DEBF0FBECDBFDF91CF911F910F91FF9033
:1038F000EF90DF90CF90BF90AF909F908F907F9090
:103900006F905F904F903F902F9008958F709270BE
:10391000892B41F0C8010E9474236BEFE62EFF242F
:10392000FA94DACFCF80D884DC24CD24DC24F12CA7
:10393000E12CC114D104D1F4C8010E9474235AEFC0
:10394000E52EFF24FA94C8CF8D85811117C0C801D8
:103950000E94BB23C8010E94BB23C8010E94BB2355
:10396000C8010E94BB23FFEFEF1AFF0A8D819E81E1
:10397000982789279827E816F906A8F441E050E02F
:10398000BE01635F7F4FC8010E94E5238D858823B8
:10399000D9F28D859FEF980F9D878823A9F2C801E2
:1039A0000E94BB23F6CFB12CA12C41E050E0BE0118
:1039B0006D5E7F4FC8010E94E5238B89982F907C14
:1039C00061F4882389F08B899FEF980F9B8B882364
:1039D00041F0C8010E94BB23F6CFC8010E94BB235F
:1039E0001B8A8B898111E1CF42E050E0BE01615F0B
:1039F0007F4FC8010E94E52342E050E0BE01635FB3
:103A00007F4FC8010E94E523C8010E94BB23C80163
:103A10000E94BB23C8010E94BB23C8010E94BB2394
:103A200042E050E0BE016F5E7F4FC8010E94E52377
:103A30008F85988981159140F9F4ED84FE84FE24E8
:103A4000EF24FE2481E0E816F104B1F489899A8913
:103A50008115944041F0C8010E94742347EFE42E81
:103A6000FF24FA9439CFB1016E5F7F4F44E050E0FC
:103A7000C8010E94E52330CFF12CE12C89899A8975
:103A8000982789279827E816F90638F4C8010E9474
:103A9000BB23FFEFEF1AFF0AF1CF2FEFA21AB20AF2
:103AA000CA14DB0409F081CFC8010E94742336EFE9
:103AB000E32EFF24FA9410CFEE24EA94FE2C0CCFD0
:103AC0009EEFE92EFF24FA9407CF8DEFE82EFF2416
:103AD000FA9402CF8F929F92AF92BF92CF92DF92D1
:103AE000EF92FF920F931F93CF93DF9300D000D0FC
:103AF00000D0CDB7DEB77C014B015A010E94001BFC
:103B00008C01892B09F06DC0F701428153816481DA
:103B1000758180915D0290915E02A0915F02B091EB
:103B20006002481759076A077B0709F45DC06701FF
:103B3000F8E0CF0ED11C0E94A92B6F7077277C5F15
:103B4000C6010E946F24813029F58FE891E09A83A5
:103B50008983F70182819381A481B5818B839C83C2
:103B6000AD83BE8345E350E0BE016F5F7F4FC6016A
:103B70000E949B23892B59F0B401C7010E94481B66
:103B8000892B29F0C6010E94A323892B31F5C60198
:103B90000E948623C80126960FB6F894DEBF0FBE9A
:103BA000CDBFDF91CF911F910F91FF90EF90DF90EC
:103BB000CF90BF90AF909F908F9008950F3F1007C8
:103BC00031F7A50168E873E1C7010E94F31B8C017E
:103BD00081E0881A910891F7DACF83E0882E912C42
:103BE000F0CF01E010E0D6CF0EEF1FEFD3CF24E0EF
:103BF00030E0AC0164E081E090E00C94882724E0A0
:103C000030E0AC0164E085E090E00C94882726E089
:103C100030E0AC0164E089E090E00C94882724E077
:103C200030E0AC0164E08FE090E00C948827AF9224
:103C3000BF92CF92DF92EF92FF920F931F93CF9399
:103C4000DF9300D000D000D0CDB7DEB76C015B01B0
:103C5000FC0182859385009711F00E94F93386E676
:103C600090E00E94F7338C0186E6F80111928A9564
:103C7000E9F7C801855B9F4F0E94A424F6011387D2
:103C80000287648581EA92E00E94E027C5010E94D4
:103C9000071E00E020E040E060E0CE0101960E94B7
:103CA0001030CE0103960E940F1E18E8E12E13E19A
:103CB000F12E00E010E020E63AEE40E050E0B501E1
:103CC000F601828593850E94AD1A8C01019709F057
:103CD0003FC0F60162857385CE0101960E94C5152D
:103CE000CE0103960E940F1EF60162857385CE01F8
:103CF00001960E94DB15CE0103960E94F71DF60186
:103D000062857385CE0101960E94D015CE0103967F
:103D10000E94FF1DF60162857385CE0101960E9407
:103D2000E6158B819C81AD81BE81F60182839383F0
:103D3000A483B583828593850E94F115F60197834C
:103D40008683828593850E94F515F6019187808789
:103D5000C80126960FB6F894DEBF0FBECDBFDF9127
:103D6000CF911F910F91FF90EF90DF90CF90BF9078
:103D7000AF9008958F929F92AF92BF92CF92DF92B1
:103D8000EF92FF920F931F93CF93DF934C015B0150
:103D90006A01E901FC01648581EA92E00E94E02762
:103DA000C5010E94071EC60102960E940F1EC8018F
:103DB00002960E94F71DC70102960E94FF1D8A818C
:103DC0009B81AC81BD81F40182839383A483B583FD
:103DD000DF91CF911F910F91FF90EF90DF90CF90E7
:103DE000BF90AF909F908F9008956F927F928F9227
:103DF0009F92AF92BF92CF92DF92EF92FF920F937A
:103E00001F93CF93DF93CDB7DEB76E970FB6F894BD
:103E1000DEBF0FBECDBF6C015B017A0149013801E5
:103E200000E02FEF4FEF6FEFCE0149960E94103068
:103E30008FE891E09A8389834B8D5C8D6D8D7E8DAB
:103E40004B835C836D837E8398878F83F3014281EC
:103E500053816481758149875A876B877C879E87E8
:103E60008D87F40142815381648175814F87588B1E
:103E7000698B7A8B9C8B8B8BF70182819381A481D8
:103E8000B5818D8B9E8BAF8BB88FCE0101967C0157
:103E90008E01095F1F4F9E01235F3F4FAE014D5EB4
:103EA0005F4FB501C6010E94BA1E6E960FB6F89418
:103EB000DEBF0FBECDBFDF91CF911F910F91FF905D
:103EC000EF90DF90CF90BF90AF909F908F907F90BA
:103ED0006F900895CF93DF93EC010E940630AE01FE
:103EE0004E5F5F4F24E030E060E08FE090E00E94A2
:103EF000CA28CE01DF91CF9108952FE831E0FC016F
:103F000031832083FB014281538164817581FC01EF
:103F1000428353836483758308950F9300E020E008
:103F200040E060E08EE792E00E94103081E692E08F
:103F30000E940630E1E6F2E0138612868AE084876A
:103F40000F91089590E080E00895DC01ED91FC91DF
:103F5000028CF38DE02D099591E089270895CF9388
:103F6000DF931F92CDB7DEB76983DC01ED91FC9141
:103F70000280F381E02D41E050E0BE016F5F7F4F92
:103F800009950F90DF91CF91089521E0FC01848580
:103F9000883009F420E0822F0895FC019485FB010C
:103FA0008485981303C081E0983009F480E0089577
:103FB000CF92DF92EF92FF920F931F93CF93DF93F5
:103FC000CDB7DEB7AF970FB6F894DEBF0FBECDBF4B
:103FD0008C016B017A01CE0101960E940630CE0160
:103FE00009960E94A424CE018A960E94063061E6BA
:103FF00072E0CE0184960E947D1FBE016C5D7F4FF2
:10400000CE0101960E94F31AAE01465D5F4FB601E4
:10401000CE0101960E946A1D81309105C1F4D8013C
:10402000ED91FC910684F785E02D8FE891E09DA34A
:104030008CA38CA59DA5AEA5BFA58EA39FA3A8A765
:10404000B9A7A701BE016C5D7F4FC8010995AF9666
:104050000FB6F894DEBF0FBECDBFDF91CF911F9199
:104060000F91FF90EF90DF90CF9008950F931F93E3
:10407000CF93DF938C01EA01FC018485883069F4D9
:1040800081E090E0F80193838283D0E0C0E0CE012C
:10409000DF91CF911F910F9108950E940B26892BDC
:1040A00079F3F5CFFC016485683021F081EA92E074
:1040B0000C94632890E080E00895CF93DF931F92E3
:1040C000CDB7DEB741E050E0BE016F5F7F4FFC012E
:1040D00084850E945C261816190634F4898190E0C4
:1040E0000F90DF91CF9108958FEF9FEFF9CFFC01F3
:1040F00084850C945C260F931F93CF93DF931F92BC
:10410000CDB7DEB78C01DC01ED91FC910084F18527
:10411000E02D0995892B79F0BE016F5F7F4FF80183
:1041200084850E94A226898190E00F90DF91CF9133
:104130001F910F9108958FEF9FEFF7CFFC018485BA
:104140000C94B026FC011382128288EE93E0A0E06A
:10415000B0E084839583A683B78385E291E0918361
:10416000808388E084870895FC011382128288EEA0
:1041700093E0A0E0B0E084839583A683B78385E2D3
:1041800091E09183808364870895FC0164856830A1
:1041900041F06295660F607E685F83E090E00C946A
:1041A000BC2780E00895CF92DF92EF92FF920F93A9
:1041B0001F93CF93DF93FC01E484F8E0EF1659F0EE
:1041C00090E080E0DF91CF911F910F91FF90EF90F1
:1041D000DF90CF9008956A018B01EC01F12C6E2DD8
:1041E00083E090E00E94BC27811123C0FC868C856F
:1041F000883031F320910A0130910B012F5F3F4F3E
:1042000011F130930B0120930A0140910A01509162
:104210000B0120E061E00E948425B8016E5F7F4FB2
:10422000A6018C850E94CE25811110C088E08C8764
:10423000C7CF8B7F8831D1F2F39420E2E20E88E081
:10424000F812CDCFD4CF20E034E0DBCFCE010E94F6
:10425000C520873151F061E070E080E090E00E947D
:10426000DA2BCE010E94C520DFCF81E090E0AACFFB
:10427000CF92DF92EF92FF92CF93DF93EC018C8588
:10428000883079F10E9404260E94A92B6B017C01E1
:10429000CE010E94C520882391F00E94A92B6C19A1
:1042A0007D098E099F09683E73408105910538F4A8
:1042B00061E070E080E090E00E94DA2BE9CFCE016F
:1042C0000E94C520882319F08C850E947625EC85F4
:1042D000F0E0EE0FFF1FE259FD4F1182108288E0DF
:1042E0008C87DF91CF91FF90EF90DF90CF90089572
:1042F000CF93DF93FC0124852830D9F0EC010E9494
:10430000C520843189F0882379F0883169F021E073
:104310008C3159F4E881F9810084F185E02DCE01DA
:10432000099521E0892B09F420E0822FDF91CF91BC
:10433000089580E0FBCF0F9300E020E040E060E0D4
:1043400084E892E00E9410300F9108950895CF9371
:10435000DF931F92CDB7DEB76983DC01ED91FC914D
:104360000280F381E02D41E050E0BE016F5F7F4F9E
:1043700009950F90DF91CF910895EF92FF920F93DF
:104380001F93CF93DF93CDB7DEB72D970FB6F89479
:10439000DEBF0FBECDBF7C0110E000E0602FCE017C
:1043A00001960E94B420CE0101960E94C520811181
:1043B00022C0F7014481558120E061E0802F0E94F6
:1043C0008425802F0E94BA25F70184819581000FF2
:1043D000111FF801E259FD4F918380832D960FB68E
:1043E000F894DEBF0FBECDBFDF91CF911F910F912B
:1043F000FF90EF9008950F5F1F4F0830110571F681
:10440000EDCFFC011382128287E491E091838083D7
:10441000758364830895AF92BF92CF92DF92EF923B
:10442000FF921F93CF93DF93CDB7DEB72D970FB6D3
:10443000F894DEBF0FBECDBF7C019EE6A92E92E0B0
:10444000B92E10E0D12CC12C612FCE0101960E9413
:10445000B420D5012D913D915D01F70184819581B5
:1044600028173907B1F4CE0101960E94C520843186
:1044700069F1CE0101960E94C5208C3151F4CE0124
:1044800001960E945220892B21F4CE0101960E94B0
:1044900038211F5F1830C1F6CD2841F4D701ED91C6
:1044A000FC910084F185E02DC70109952D960FB68A
:1044B000F894DEBF0FBECDBFDF91CF911F91FF906B
:1044C000EF90DF90CF90BF90AF900895CC24C3942D
:1044D000D12CDFCF7F928F929F92AF92BF92CF92DB
:1044E000DF92EF92FF920F931F93CF93DF93CDB79D
:1044F000DEB72D970FB6F894DEBF0FBECDBF6C01AF
:104500005B014A010E940B228EE6E82E82E0F82E23
:10451000712C10E000E0672DCE0101960E94B420BE
:10452000F701219131917F01F6018481958128174E
:10453000390771F4CE0101960E94C520873141F4FC
:10454000A401B501CE0101960E943620080F191F63
:104550007394F8E07F12DFCFC8012D960FB6F89460
:10456000DEBF0FBECDBFDF91CF911F910F91FF90A6
:10457000EF90DF90CF90BF90AF909F908F907F9003
:104580000895AF92BF92CF92DF92FF920F931F9345
:10459000CF93DF93CDB7DEB72D970FB6F894DEBF7C
:1045A0000FBECDBF8C015B01CB010E940B228EE6BA
:1045B000C82E82E0D82EF12C6F2DCE0101960E94DC
:1045C000B420F601219131916F01F501848195812B
:1045D00028173907F1F5CE0101960E94C5208731D1
:1045E00091F5CE0101960E945220892B91F18B8189
:1045F0009C81F801938382838D819E81AF81B885F0
:1046000084839583A683B78389859A85AB85BC858A
:1046100080879187A287B38785E291E09183808329
:104620008D858487C8012D960FB6F894DEBF0FBE26
:10463000CDBFDF91CF911F910F91FF90DF90CF9071
:10464000BF90AF900895CE0101960E94C5208C3195
:1046500041F2F394F8E0FF12AFCF68E0C8010E9486
:10466000B420E0CF0F9300E020E040E060E08AE873
:1046700092E00E9410300F91089580E00895DC01CF
:10468000ED91FC91048CF58DE02D09942FE831E03B
:10469000FC0131832083FB0141895289638974893C
:1046A000FC0142835383648375830895FC018589EB
:1046B00096890895FC01818D928D0895CF93DF93A3
:1046C0001F92CDB7DEB76983DC01ED91FC910280CA
:1046D000F381E02D41E050E0BE016F5F7F4F09950F
:1046E0000F90DF91CF910895CF93DF93EC01898DE7
:1046F0009A8D892B41F0E881F9810284F385E02DC0
:10470000CE010995F4CFDF91CF910895CF93DF9338
:10471000EC018C85883061F00E947625EC85F0E014
:10472000EE0FFF1FE259FD4F1182108288E08C8747
:10473000DF91CF910895FC01108E178A6E5F7F4F35
:1047400084850C94DF26FC0184850C940427CF9388
:10475000DF93EC019A018F89988DAB01BC018C85A8
:104760000E94B1262F89388D280F391F388F2F8B43
:10477000DF91CF9108950F931F93CF93DF931F92F3
:10478000CDB7DEB7FC01218D328D232B41F48FEFA5
:104790009FEF0F90DF91CF911F910F9108958C01A2
:1047A00041E050E0BE016F5F7F4FFC0184850E94B5
:1047B0005C26181619065CF7F801818D928D019719
:1047C000928F818F898190E0E4CFCF93DF93FC01BA
:1047D000218D328D2115310529F48FEF9FEFDF9167
:1047E000CF910895EC0184854217530708F0A90181
:1047F0000E945C261816190684F7298D3A8D281B0D
:10480000390B3A8F298FEBCFCF93DF931F92CDB720
:10481000DEB7FC01218D328D8FEF9FEF232B41F00E
:10482000BE016F5F7F4F84850E94A226898190E040
:104830000F90DF91CF9108950F931F93CF93DF9344
:10484000CDB7DEB728970FB6F894DEBF0FBECDBF49
:104850008C01DC01ED91FC910680F781E02D09953A
:10486000F801648581EA92E00E946328892BA1F116
:1048700048E050E0BE016F5F7F4FD8011C968C91DD
:104880000E945C2618161906E4F4BE016F5F7F4F84
:10489000C8010F960E9428308D8190E0982F8827BC
:1048A0002E81820F911DF801968B858B8F81282F89
:1048B00030E0322F22278885820F932F911D928F0F
:1048C000818F28960FB6F894DEBF0FBECDBFDF9163
:1048D000CF911F910F91089590E080E0F2CFEF9279
:1048E000FF920F931F93CF93DF93FC01E484F8E0D2
:1048F000EF1641F080E0DF91CF911F910F91FF9073
:10490000EF9008958B01EC01F12C6E2D83E090E087
:104910000E94BC2781110FC0FC868C85883051F322
:104920001E870D871A8E198E20E0A80162E00E9472
:10493000842581E0E0CF883179F3F39420E2E20E20
:1049400088E0F812E2CFE9CFFC011382128288EEF0
:1049500093E0A0E0B0E084839583A683B78385E5E8
:1049600091E09183808388E08487CF010F960C9437
:104970000630CF92DF92EF92FF920F931F93CF9367
:10498000DF93CDB7DEB7AF970FB6F894DEBF0FBE9B
:10499000CDBF8C016B017A01CE0101960E940630D9
:1049A000CE0109960E94A424CE018A960E94063068
:1049B00061E672E0CE0184960E947D1FBE016C5DAF
:1049C0007F4FCE0101960E94F31AAE01465D5F4F04
:1049D000B601CE0101960E946A1D81309105C1F495
:1049E000D801ED91FC910488F589E02D8FE891E0E4
:1049F0009DA38CA38CA59DA5AEA5BFA58EA39FA3AB
:104A0000A8A7B9A7A701BE016C5D7F4FC801099592
:104A1000AF960FB6F894DEBF0FBECDBFDF91CF913A
:104A20001F910F91FF90EF90DF90CF9008950F931B
:104A300000E020E040E060E080E992E00E94103079
:104A40000F9108950F9300E020E040E060E086E9D8
:104A500092E00E9410300F910895AB018295880F6B
:104A6000807E6CE0680F24E030E08CE090E00C94F5
:104A700088279B018295880F807E68E0680FC901B6
:104A80000C94BC2762E070E00C9439259B01829560
:104A9000880F807E6CE0680FC9010C946227CF9369
:104AA000DF93C82FD62F472F64E070E00E94462581
:104AB0004D2F65E070E08C2FDF91CF910C9446254F
:104AC000462F62E070E00C944625CF93DF93C82F09
:104AD000D62F472F60E170E00E9446254D2F61E1FF
:104AE00070E08C2FDF91CF910C944625CF93C82F87
:104AF00040E150E0682F81EA92E00E9469296FEF5F
:104B00008C2FCF910C946025FF920F931F93CF931E
:104B1000DF939FEF960F953058F5F22E8A01D62F2E
:104B2000C82F0E9476254D2F4F2970E060E08C2F12
:104B30000E944625B801012B51F460919C027091AE
:104B40009D026F5F7F4F70939D0260939C028C2F3C
:104B50000E944F2541E050E06C2F81EA92E00E94D4
:104B6000692981E0DF91CF911F910F91FF90089506
:104B700080E0F8CFCF93C82F63E070E00E94392522
:104B8000833151F442E050E06C2F81EA92E00E94C0
:104B9000692981E0CF91089580E0FCCF0F931F93A6
:104BA000CF93FB0190819F3F59F491819F3F99F4EE
:104BB00092819F3F81F493819F3F69F490E01FC0F1
:104BC000911109C09181911106C09281911103C088
:104BD00093819923A1F04115510581F38A01BF0109
:104BE000C82F0E942D25B8018C2F0E94652544E016
:104BF00050E06C2F81EA92E00E94692991E0892FB0
:104C0000CF911F910F91089548E050E0682F81EAFD
:104C100092E00C946929CF92DF92EF92FF920F936A
:104C20001F93CF93C82F7B018A014130584010F069
:104C300000E018E06C2F81EA92E00E942F286C01BE
:104C400063E070E08C2F0E943925873111F08C31A0
:104C500059F5C016D10670F39801A7016C2F81EAAF
:104C600092E00E94BF2840E250E06C2F81EA92E07F
:104C70000E9469298C2F0E94422584FD18C063E0A0
:104C800070E08C2F0E9439258111F4CF8C2F0E9467
:104C9000762510E000E0C801CF911F910F91FF90A1
:104CA000EF90DF90CF90089510E000E0D5CF60E165
:104CB0008C2F0E946025EFCFCF92DF92EF92FF9270
:104CC0000F931F93CF93DF93182F6B017A01682FF7
:104CD00081EA92E00E946328EC010097E1F463E02E
:104CE00070E0812F0E943925843159F0882349F0E2
:104CF000C1E0D0E08C3111F4D0E0C0E0D195C19595
:104D0000D109CE01DF91CF911F910F91FF90EF90CC
:104D1000DF90CF900895E816F9060CF4E7011C1611
:104D20001D067CF700E09E01A601612F81EA92E05A
:104D30000E94182940E450E0612F81EA92E00E942D
:104D40006929DFCF0F93AB0101E021E030E0682F4C
:104D500081EA92E00E94182981E090E00F91089585
:104D60000895AF92BF92CF92DF92FF920F931F935D
:104D7000CF93DF93F82E6B015A01E901682F81EA86
:104D800092E00E942F288C179D0730F46F2D81EA46
:104D900092E00E942F28EC018E019501A6016F2D53
:104DA00081EA92E00E947F28CE01DF91CF911F918E
:104DB0000F91FF90DF90CF90BF90AF9008950F9329
:104DC0001F93CF93FB019081911109C091819111A3
:104DD00006C09281911103C09381992391F04115EE
:104DE000510579F08A01BF01C82F0E942D25B80115
:104DF0008C2F0E94652581E090E0CF911F910F914B
:104E0000089590E080E0F9CFCF93C82F40E250E0C2
:104E1000682F81EA92E00E9469298C2F0E94422526
:104E200084FD0DC08C2F0E94422583FFF6CF68E1E0
:104E30008C2F0E94602590E080E0CF91089560E182
:104E40008C2F0E94602581E090E0F7CF20915302E3
:104E5000222381F03FB7F89420915302213069F466
:104E60002DB3209351024DB320915202209524235B
:104E70002DBB3FBF8CBD9DBD089530935102FACF2D
:104E80008EBD00000DB407FEFDCF8EB50895809154
:104E90005302882361F09FB7F894209153028091C8
:104EA0005102213019F48DBB9FBF08958FBF089523
:104EB00060E080919E020C94872D61E080919E02BB
:104EC0000C94872D0F931F93CF93DF93182F092FE7
:104ED000D62FC42F80919F029091A0020E94262776
:104EE0000E945827802F0E944027812F0E94402730
:104EF0008D2F0E9440278C2F0E9440270E945D2703
:104F00000E94472781E0DF91CF911F910F91089573
:104F1000DF92EF92FF920F931F93CF93DF93D82FDF
:104F2000D92EC62F7A01890180919F029091A0020B
:104F30000E9426270E9458278D2D0E9440278D2FE2
:104F40000E9440278C2F0E944027E701E00EF11EAF
:104F5000CE15DF0521F089910E944027F9CF0E94EC
:104F60005D270E944727C801DF91CF911F910F91C4
:104F7000FF90EF90DF9008951F93CF93DF93D82F8A
:104F8000192FC62F80919F029091A0020E94262780
:104F90000E945827812F0E9440278D2F0E94402772
:104FA0008C2F0E94402780E00E944027C82F0E943B
:104FB0005D270E9447278C2FDF91CF911F91089585
:104FC0000F931F93CF9360939E0268EE73E080E08F
:104FD00090E00E94DA2B61E080919E020E944B2DAE
:104FE0000E94881560E090E080E00E94BC27482F76
:104FF000406864E090E080E00E946227CCE008E036
:1050000010E042E06C2F8EE190E00E94622742E0C7
:105010006C2F8FE190E00E94622701501109C05E61
:105020000115110571F7CF911F910F9108951F93ED
:10503000CF93DF93182F60E270E00E943925C82FCC
:10504000D0E0DC2FCC2761E270E0812F0E9439256F
:105050008C0F9D2F911DDF91CF911F910895FF928D
:105060000F931F93CF93DF93F62ED0E0C0E08F2DE8
:105070000E9417288C01892B21F08F2D0E94172860
:10508000EC01C017D10799F7CE01DF91CF911F91A5
:105090000F91FF9008951F93CF93DF93182F66E22F
:1050A00070E00E943925C82FD0E0DC2FCC2767E2C2
:1050B00070E0812F0E9439258C0F9D2F911DDF916B
:1050C000CF911F910895FF920F931F93CF93DF937A
:1050D000F62ED0E0C0E08F2D0E944B288C01892B4A
:1050E00021F08F2D0E944B28EC01C017D10799F7B2
:1050F000CE01DF91CF911F910F91FF900895BF9244
:10510000CF92DF92EF92FF920F931F93CF93DF9393
:10511000B62E7A01690164E270E08B2D0E94392578
:10512000C82F65E270E08B2D0E943925D0E0DC2F7E
:10513000CC278E0D9F2D911DC80FD91F6B2D629509
:10514000660F607E6C5E9801A601CE010E948827E2
:105150000C0F1D1F412F64E270E08B2D0E9446252D
:10516000402F65E270E08B2DDF91CF911F910F9161
:10517000FF90EF90DF90CF90BF900C9446250F9357
:105180001F9389019A0150E040E00E947F281F91FF
:105190000F910895DF92EF92FF920F931F93CF9399
:1051A000DF93D82FD92EC62F7A01890180919F02D3
:1051B0009091A0020E9426270E9458278D2D0E94C0
:1051C00040278D2F0E9440278C2F0E944027E70107
:1051D000E00EF11ECE15DF0529F080E00E94402789
:1051E0008993F8CF0E945D270E944727C801DF916D
:1051F000CF911F910F91FF90EF90DF9008950F9343
:105200001F93CF93DF9300D0CDB7DEB75A83498386
:10521000A901980189819A816295660F607E685E16
:105220000F900F90DF91CF911F910F910C94CA288E
:105230008F929F92AF92BF92CF92DF92EF92FF92A6
:105240000F931F93CF93DF936C01962E5A01790130
:10525000802E68E270E0892D0E943925C82FD0E0A9
:10526000DC2FCC2769E270E0892D0E943925C80F18
:10527000D11D87019501AE01692DC6010E94FF284D
:1052800081101AC0CE0DDF1D4D2F68E270E0892D10
:105290000E9446254C2F69E270E0892DDF91CF9165
:1052A0001F910F91FF90EF90DF90CF90BF90AF9044
:1052B0009F908F900C944625DF91CF911F910F9175
:1052C000FF90EF90DF90CF90BF90AF909F908F9026
:1052D0000895CF93C62F61E070E08C2F0E94462581
:1052E00061E070E08C2F0E9439258111F9CFCF91B8
:1052F0000895EFE9F2E080E5808381E081830895FD
:10530000FF920F931F93CF93DF93FC011081C18114
:10531000D281F8948981012F009580238983789424
:105320008DE7F82EFA94FF2061F182E090E00E9470
:10533000132C88818123B1F3F8948A8180238A8396
:105340008981812B8983789480EE91E00E94132CCF
:10535000F89489818023898386E490E00E94132C4D
:1053600088811823C1E009F0C0E078948AE991E0CF
:105370000E94132C8C2FDF91CF911F910F91FF90E2
:105380000895C0E0F7CF1F93CF93DF93FC01108106
:10539000C181D281912F909560FF16C0F8948A81C7
:1053A00089238A838981812B89838AE090E00E9406
:1053B000132C8A81182B1A83789487E390E0DF916D
:1053C000CF911F910C94132CF8948A8189238A839E
:1053D0008981812B898381E490E00E94132C8A814A
:1053E000182B1A83789485E090E0E9CF0F931F93F0
:1053F000CF93DF93FC011081C181D281F894898120
:10540000812B89838A81012F009580238A8383E001
:1054100090E00E94132C8981802389838AE090E0A8
:105420000E94132CC881789485E390E00E94132C8D
:10543000C12381E009F480E0DF91CF911F910F91AA
:105440000895DF92EF92FF920F931F93CF93DF9314
:10545000EC01D62EE42E08E010E0FF24F39461E086
:105460008D2D8F2109F460E0CE010E94C329FF0C2D
:1054700001501109A1F7E11010C0F894E981FA81F7
:1054800091818881809589238183E981FA81928144
:1054900088818095892382837894DF91CF911F91B1
:1054A0000F91FF90EF90DF900895EF92FF920F938E
:1054B0001F93CF93DF937C0108E010E0C0E0D1E0C0
:1054C000C7010E94F6298111CD2BDD0F0150110972
:1054D000B9F78C2FDF91CF911F910F91FF90EF9033
:1054E0000895EF92FF920F931F93CF93DF938C0158
:1054F0007B0140E065E50E94212AE70188E0E80E93
:10550000F11C699140E0C8010E94212ACE15DF05F7
:10551000C1F7DF91CF911F910F91FF90EF90089508
:1055200040E06CEC0C94212AFC011386158614864D
:1055300012861186108617821682158214821382B3
:1055400008951F93CF93DF93EC01162F60E0812F16
:105550000E944B2D612F70E0FB01E651FB4FE4915F
:10556000E883FB01EE5FFA4FE491F0E0EE0FFF1FDE
:10557000E65EFA4F859194919A838983CE01DF91FB
:10558000CF911F910C94942ABF92CF92DF92EF9209
:10559000FF920F931F93CF93DF93EC01B62EC72E8C
:1055A000142F8D85811105C0CE010E9480298111A3
:1055B0000EC01B861D861C8680E0DF91CF911F9157
:1055C0000F91FF90EF90DF90CF90BF90089540E053
:1055D00060EF111101C06CEECE010E94212A01E0A2
:1055E000E12CD12C11E0CE010E94F629F82ECE013B
:1055F0000E94F62991E0F91218C0813099F5113412
:10560000C0F2DB86D11002C081E08D878B818823B8
:1056100081F22396EB2DFC2DCF0108962991219341
:10562000E817F907D9F781E0C8CFEE2DF0E0F812BE
:105630000FC08B851817A0F4DE01AE0FBF1F1396A5
:105640008C91802379F4F12C193008F41C87D12E29
:10565000EC0FFD1F8381902F9095892383830AC0CF
:105660008113F1CFFE01EE0DF11D8381802B838329
:10567000FF24F3946F2DCE010E94C3291F5F000FFA
:1056800011F4E39401E087E08E1508F0ACCFB7CFBA
:10569000DC0180E0615090F09D919827E92FEF7038
:1056A000F0E0EE54FB4F2491E92FE295EF70F0E02B
:1056B000EE53FB4FE491822F8E27ECCF08951F927B
:1056C0000F920FB60F9211242F933F938F939F93B6
:1056D000AF93BF938091A3029091A402A091A502E1
:1056E000B091A6023091A20226E0230F2D3758F583
:1056F0000296A11DB11D2093A2028093A302909354
:10570000A402A093A502B093A6028091A702909153
:10571000A802A091A902B091AA020196A11DB11DF3
:105720008093A7029093A802A093A902B093AA0223
:10573000BF91AF919F918F913F912F910F900FBE8D
:105740000F901F90189529E8230F0396A11DB11DF6
:10575000D2CF2FB7F8946091A3027091A4028091E8
:10576000A5029091A6022FBF08953FB7F8948091AB
:10577000A7029091A802A091A902B091AA0226B511
:10578000A89B05C02F3F19F00196A11DB11D3FBF79
:10579000BA2FA92F982F8827BC01CD01620F711D48
:1057A000811D911D43E0660F771F881F991F4A9541
:1057B000D1F708958F929F92AF92BF92CF92DF92CE
:1057C000EF92FF926B017C010E94B52B4B015C01B3
:1057D000C114D104E104F104E9F00E94FB330E94FA
:1057E000B52B681979098A099B09683E73408105C0
:1057F000910570F321E0C21AD108E108F10888EEA2
:10580000880E83E0981EA11CB11CC114D104E104D0
:10581000F10429F7FF90EF90DF90CF90BF90AF9009
:105820009F908F9008958330910528F0880F991FDD
:1058300004970197F1F70895789484B5826084BD48
:1058400084B5816084BD85B5826085BD85B5816084
:1058500085BDEEE6F0E0808181608083E1E8F0E0E4
:105860001082808182608083808181608083E0E813
:10587000F0E0808181608083E1EBF0E080818460F2
:105880008083E0EBF0E0808181608083E1E9F0E0FB
:10589000808182608083808181608083E0E9F0E0A4
:1058A000808181608083E1EAF0E080818260808392
:1058B000808181608083E0EAF0E080818160808384
:1058C000EAE7F0E080818460808380818260808369
:1058D00080818E7F80838081806880831092C10068
:1058E00008951F93CF93DF93182FEB0161E00E947F
:1058F0004B2D209739F460E0812FDF91CF911F91DC
:105900000C94872DCF3FD10511F461E0F5CFE12F45
:10591000F0E0EE52FB4FE491E150ED3008F070C042
:10592000F0E0EB56F34D0C948D36A22CAA2CAF2C44
:10593000B92C002D002DC32CCB2CD32CDD2C002D0D
:10594000E72CF62C84B5806884BDC7BDDF91CF916C
:105950001F91089584B5806284BDC8BDF7CF809142
:105960008000806880938000D0938900C093880075
:10597000EDCF80918000806280938000D0938B0077
:10598000C0938A00E3CF8091B00080688093B0001C
:10599000C093B300DBCF8091B00080628093B000F1
:1059A000C093B400D3CF8091900080688093900022
:1059B000D0939900C0939800C9CF809190008062E5
:1059C00080939000D0939B00C0939A00BFCF8091AA
:1059D000A00080688093A0008091A0008F7B8093BE
:1059E000A000D093A900C093A800B0CF8091A000E0
:1059F00080628093A000D093AB00C093AA00A6CF92
:105A0000C038D1050CF081CF76CF81508D3008F0B1
:105A10003DC0E82FF0E0E15FF24D0C948D36262D6D
:105A20002A2D1C2D222D462D462D2D2D332D372D83
:105A30003D2D462D412D472D809180008F778093FD
:105A400080000895809180008F7DF9CF84B58F7795
:105A500084BD089584B58F7DFBCF8091B0008F7792
:105A60008093B00008958091B0008F7DF9CF809130
:105A700090008F77809390000895809190008F7DA3
:105A8000F9CF8091A0008F778093A0000895809136
:105A9000A0008F7DF9CFCF93DF9390E0FC01E6511A
:105AA000FB4F24918E5F9A4FFC0184918823C9F0AB
:105AB00090E0880F991FFC01EE5CFA4FA591B4911C
:105AC000FC01EA5DFA4FC591D49161110DC09FB7F9
:105AD000F8948C91209582238C93888128232883A5
:105AE0009FBFDF91CF910895623051F49FB7F89432
:105AF0003C91822F809583238C93E8812E2BEFCFCE
:105B00008FB7F894EC912E2B2C938FBFEACF1F9375
:105B1000CF93DF93282F30E0F901EE52FB4F8491B1
:105B2000F901E651FB4FD491F901EE5FFA4FC491B0
:105B3000CC23A9F0162F81110E94052DEC2FF0E047
:105B4000EE0FFF1FEA5DFA4FA591B4918FB7F8945D
:105B5000EC91111108C0D095DE23DC938FBFDF914B
:105B6000CF911F910895DE2BF8CFCF93DF93282F8D
:105B700030E0F901EE52FB4F8491F901E651FB4F01
:105B8000D491F901EE5FFA4FC491CC23A1F08111B9
:105B90000E94052DEC2FF0E0EE0FFF1FE65EFA4F9E
:105BA000A591B491EC91ED2381E090E009F480E0BF
:105BB000DF91CF91089580E090E0FACFFC01918DC4
:105BC000228D892F90E081509F4F821B91096FEFAA
:105BD00070E00E9438360895FC01918D828D9817EF
:105BE00031F0828DE80FF11D858D90E008958FEFE3
:105BF0009FEF0895FC01918D828D981781F0A28D01
:105C0000AE0FBF2FB11D5D968C91228D2F5F91E05D
:105C10002F3F08F490E0920F928F90E008958FEF5D
:105C20009FEF0895FC01538D448D252F30E0842F84
:105C300090E0821B930B541710F0CF9608950197B4
:105C400008958DE89FE2892B49F080E090E0892B50
:105C500029F00E948D2F81110E94000080E090E0C9
:105C6000892B49F080E090E0892B29F00E94000008
:105C700081110C9400000895FC01A48DA80FB92F88
:105C8000B11DA45EBE4F2C91848D90E001968F7360
:105C90009927848FA689B7892C93A089B1898C9183
:105CA000837080648C93938D848D981306C00288D2
:105CB000F389E02D80818F7D80830895CF93DF93DA
:105CC000EC01888D8823B9F0AA89BB89E889F98914
:105CD0008C9185FD03C0808186FD0DC00FB607FC49
:105CE000F7CF8C9185FFF2CF808185FFEDCFCE017C
:105CF0000E943C2EE9CFDF91CF910895EF92FF9261
:105D00000F931F93CF93DF93EC0181E0888F9B8DDE
:105D10008C8D98131AC0E889F989808185FF15C098
:105D20009FB7F894EE89FF896083E889F9898081BB
:105D30008370806480839FBF81E090E0DF91CF918A
:105D40001F910F91FF90EF900895F62E0B8D10E0AC
:105D50000F5F1F4F0F731127E02E8C8D8E110CC01B
:105D60000FB607FCFACFE889F989808185FFF5CF66
:105D7000CE010E943C2EF1CFEB8DEC0FFD2FF11DDB
:105D8000E45EFE4FF0829FB7F8940B8FEA89FB899F
:105D900080818062CFCFCF92DF92EF92FF921F93EC
:105DA000CF93DF93EC016A017B01122F60E874E866
:105DB0008EE190E0A70196010E944C3621503109F6
:105DC000410951095695479537952795E889F989ED
:105DD00082E08083211580E1380798F0E889F9890D
:105DE000108260E472E48FE090E0A70196010E94C7
:105DF0004C3621503109410951095695479537953F
:105E00002795EC85FD853083EE85FF852083188EF0
:105E1000EC89FD891083EA89FB8980818061808318
:105E2000EA89FB89808188608083EA89FB89808197
:105E300080688083EA89FB8980818F7D8083DF9100
:105E4000CF911F91FF90EF90DF90CF9008951F9218
:105E50000F920FB60F9211242F935F936F937F933E
:105E60008F939F93AF93BF93EF93FF93E091BB0208
:105E7000F091BC028081E091C102F091C20282FDEA
:105E800024C020818091C40290E001966FEF70E001
:105E90000E9438369091C502981741F0E091C402F3
:105EA000F0E0E555FD4F258F8093C402FF91EF91FF
:105EB000BF91AF919F918F917F916F915F912F9142
:105EC0000F900FBE0F901F9018958081EFCF1F92FB
:105ED0000F920FB60F9211242F933F934F935F931E
:105EE0006F937F938F939F93AF93BF93EF93FF93A2
:105EF0008BEA92E00E943C2EFF91EF91BF91AF910F
:105F00009F918F917F916F915F914F913F912F91D1
:105F10000F900FBE0F901F9018958BEA92E00E9491
:105F2000DE2D21E0892B09F420E0822F0895EBEA91
:105F3000F2E01382128288EE93E0A0E0B0E0848366
:105F40009583A683B7838DE791E09183808385EC69
:105F500090E09587848784EC90E09787868780EC33
:105F600090E0918B808B81EC90E0938B828B82EC24
:105F700090E0958B848B86EC90E0978B868B118ECE
:105F8000128E138E148E08958F929F92AF92BF92AD
:105F9000CF92DF92EF92FF920F931F93CF93DF93F5
:105FA0007C018B014C0182E0880E911C5701E5E0D9
:105FB000AE0EB11CD0E0C0E0F40161914F014AE0A7
:105FC00050E0C8010E9472316C016EE2C8010E946B
:105FD00091308C0D9D1DC80FD91F8A149B0461F749
:105FE0004AE050E0F7016581C8010E9472318C0FD0
:105FF0009D1FDF91CF911F910F91FF90EF90DF9048
:10600000CF90BF90AF909F908F9008952FE831E090
:10601000FC01318320831282138214821582089539
:106020000F93FC018FE891E0918380836283438327
:10603000248305830F910895DC018FE891E08D930F
:106040009D9384E0FB0101900D928A95E1F70895FC
:10605000DC01129624E0FB0101900D922A95E1F7F4
:106060000895AF92BF92CF92DF92EF92FF920F937B
:106070001F93CF93DF936C017B018B01040F151FDE
:10608000EB015E01AE18BF08C017D10759F0699146
:10609000D601ED91FC910190F081E02DC6010995AA
:1060A000892B79F7C501DF91CF911F910F91FF9057
:1060B000EF90DF90CF90BF90AF900895FB010190DB
:1060C0000020E9F73197AF01461B570BDC01ED913A
:1060D000FC910280F381E02D0994EF92FF920F93DF
:1060E0001F93CF93DF938C017B01D0E0C0E0F701D9
:1060F000EC0FFD1F6491662361F0D801ED91FC91D6
:106100000190F081E02DC8010995892B11F02196AD
:10611000EECFCE01DF91CF911F910F91FF90EF90C5
:106120000895DC01ED91FC910190F081E02D09943E
:10613000DB01ED91FC9111970190F081E02DBC0104
:10614000CD01099461E971E00C945E300F931F93C7
:10615000CF93DF93EC010E946D308C01CE010E9441
:10616000A230800F911FDF91CF911F910F91089561
:106170008F929F92AF92BF92EF92FF920F931F93D5
:10618000CF93DF93CDB7DEB7A1970FB6F894DEBFFC
:106190000FBECDBF7C01FA01CB0119A2223008F459
:1061A0002AE08E010F5D1F4F822E912CB12CA12C65
:1061B000BF01A50194010E944C36F901CA016A3061
:1061C0000CF5605DD8016E938D01232B242B252BBC
:1061D00079F790E080E0109721F0BD01C7010E949F
:1061E0005E30A1960FB6F894DEBF0FBECDBFDF9133
:1061F000CF911F910F91FF90EF90BF90AF909F9024
:106200008F900895695CDECFCF92DF92EF92FF927C
:106210000F931F93CF93DF932115310581F4DC0198
:10622000ED91FC910190F081E02D642FDF91CF91F1
:106230001F910F91FF90EF90DF90CF9009942A303B
:10624000310501F52AE077FF1DC06A017B01EC01F1
:106250006DE20E9491308C0144275527BA014C19F8
:106260005D096E097F092AE0CE010E94B830800FD7
:10627000911FDF91CF911F910F91FF90EF90DF90D1
:10628000CF900895DF91CF911F910F91FF90EF90E4
:10629000DF90CF900C94B8309A01AB01770F660B6A
:1062A000770B0C9404310F931F93CF93DF93EC0182
:1062B0000E944C318C01CE010E94A230800F911FB0
:1062C000DF91CF911F910F9108952115310541F470
:1062D000DC01ED91FC910190F081E02D642F099497
:1062E0000C94B8309A01462F50E070E060E00C94B6
:1062F00065310F931F93CF93DF93EC010E947231AE
:106300008C01CE010E94A230800F911FDF91CF91AE
:106310001F910F9108959A01AB0170E060E00C9419
:1063200065310F931F93CF93DF93EC010E9465318A
:106330008C01CE010E94A230800F911FDF91CF917E
:106340001F910F9108952F923F924F925F926F92FB
:106350007F928F929F92AF92BF92CF92DF92EF92F5
:10636000FF921F93CF93DF93EC016A017B01722EA2
:10637000AB019601CB01B6010E94333664E971E0AE
:10638000811126C046015701E894B7F82FEF3FEF7F
:106390004FE75FE7C501B4010E94333681110CC09D
:1063A0002FEF3FEF4FE75FE7C501B4010E9469346B
:1063B00068E971E0181664F02FEF3FEF4FE75FE4F4
:1063C000C701B6010E94C1351816B4F46CE971E03A
:1063D000CE01DF91CF911F91FF90EF90DF90CF9092
:1063E000BF90AF909F908F907F906F905F904F90F5
:1063F0003F902F900C945E302FEF3FEF4FE75FEC14
:10640000C701B6010E94693487FDE0CF20E030E08B
:10641000A901C701B6010E946934312C212C87FFE4
:1064200009C06DE2CE010E9491301C01F7FAF09490
:10643000F7F8F09410E060E070E080E09FE3711600
:1064400041F020E030E040E251E40E946E341F5FF2
:10645000F6CFA70196010E94FD332B013C010E945B
:10646000E0344B015C012AE0BC01A401CE010E9492
:10647000B8307C01E20CF31C1123B1F1C501B40169
:106480000E940F359B01AC01C301B2010E94FC3395
:106490004B015C016EE2CE010E949130E80EF91EC4
:1064A000115010F120E030E040E251E4C501B401A8
:1064B0000E94C6352B013C010E94E0344B014AE0AA
:1064C00050E0CE010E948B31E80EF91EB40190E03D
:1064D00080E00E940F359B01AC01C301B2010E9414
:1064E000FC334B015C01DCCFC701DF91CF911F91E1
:1064F000FF90EF90DF90CF90BF90AF909F908F90E4
:106500007F906F905F904F903F902F9008950C94E4
:10651000A3310F931F93CF93DF93EC010E94A92B1C
:10652000688779878A879B87E881F9810284F38568
:10653000E02DCE01099597FF15C00E94A92B088573
:1065400019852A853B85601B710B820B930B0C818F
:106550001D812E813F81601771078207930720F309
:106560008FEF9FEFDF91CF911F910F9108950F93C0
:106570001F93CF93DF93EC010E94A92B6887798743
:106580008A879B87E881F9810484F585E02DCE0117
:10659000099597FF15C00E94A92B088519852A85A2
:1065A0003B85601B710B820B930B0C811D812E812F
:1065B0003F81601771078207930720F38FEF9FEFEA
:1065C000DF91CF911F910F910895FF920F931F9329
:1065D000CF93DF93EC018B01F42ECE010E94B732F2
:1065E00097FD1DC08D329105D1F09C0120533109DA
:1065F0002A303105A0F0FF2019F08E32910579F094
:106600000130110551F00230110589F48D309105EA
:1066100071F05CF40997029750F08FEF9FEFDF91D4
:10662000CF911F910F91FF9008958097B1F7E88166
:10663000F9810284F385E02DCE010995CECFFC01CE
:1066400044835583668377830895BF92CF92DF9208
:10665000EF92FF920F931F93CF93DF938C01C42F80
:1066600040E00E94E532FC01C12CD12C760197FD5F
:106670003EC0B12C0C2E000CDD0BCE17DF07D9F07D
:10668000ED32F10509F43FC0CF01C0970A9798F4A5
:10669000AAE0B0E0A70196010E949A366F01FF0FB1
:1066A000EE08FF08C60ED71EE81EF91E80E3C81AC2
:1066B000D108E108F108D801ED91FC910284F3853D
:1066C000E02DC8010995C8010E94B732FC01C097AE
:1066D0000A9798F2CE17DF0781F2BB2041F0F094C1
:1066E000E094D094C094C11CD11CE11CF11CC701E2
:1066F000B601DF91CF911F910F91FF90EF90DF9046
:10670000CF90BF900895BB24B394D5CFAF92BF92E2
:10671000CF92DF92EF92FF920F931F93CF93DF936D
:106720005C017B018B01040F151FEB016E01CE187C
:10673000DF08C017D10739F0C5010E94893297FDE3
:1067400002C08993F3CFC601DF91CF911F910F91C2
:10675000FF90EF90DF90CF90BF90AF900895CF92D1
:10676000DF92EF92FF926B017C01C114D104E1042E
:10677000F10441F00E942538A70196010E946E366F
:106780006B017C01C701B601FF90EF90DF90CF90C5
:106790000895CF92DF92EF92FF926B017C01C216B7
:1067A000D306E406F50664F4CA01B9016C197D0943
:1067B0008E099F090E94AF33C60ED71EE81EF91E30
:1067C000C701B601FF90EF90DF90CF900895089534
:1067D0000E941C2C0E94E7330E94FA10C1E2DEE204
:1067E0000E94D5142097E1F30E94212EF9CF0C943A
:1067F000B4360C94503708955058BB27AA270E94EE
:1068000014340C9487350E94793538F00E94803515
:1068100020F039F49F3F19F426F40C9476350EF4E9
:10682000E095E7FB0C947035E92F0E94983558F3FA
:10683000BA17620773078407950720F079F4A6F565
:106840000C94BA350EF4E0950B2EBA2FA02D0B0147
:10685000B90190010C01CA01A0011124FF27591BA5
:1068600099F0593F50F4503E68F11A16F040A22FAB
:10687000232F342F4427585FF3CF4695379527951C
:10688000A795F0405395C9F77EF41F16BA0B620B1B
:10689000730B840BBAF09150A1F0FF0FBB1F661F62
:1068A000771F881FC2F70EC0BA0F621F731F841FA5
:1068B00048F4879577956795B795F7959E3F08F0CB
:1068C000B0CF9395880F08F09927EE0F979587958D
:1068D00008950E944C3508F481E008950E948234A6
:1068E0000C9487350E94803558F00E94793540F02D
:1068F00029F45F3F29F00C94703551110C94BB358D
:106900000C9476350E94983568F39923B1F355239A
:1069100091F3951B550BBB27AA27621773078407B2
:1069200038F09F5F5F4F220F331F441FAA1FA9F348
:1069300035D00E2E3AF0E0E832D091505040E69536
:10694000001CCAF72BD0FE2F29D0660F771F881F97
:10695000BB1F261737074807AB07B0E809F0BB0B8A
:10696000802DBF01FF2793585F4F3AF09E3F51059E
:1069700078F00C9470350C94BB355F3FE4F3983E8F
:10698000D4F3869577956795B795F7959F5FC9F787
:10699000880F911D9695879597F90895E1E0660F08
:1069A000771F881FBB1F621773078407BA0720F081
:1069B000621B730B840BBA0BEE1F88F7E0950895EA
:1069C0000E94A03588F09F5798F0B92F9927B751AA
:1069D000B0F0E1F0660F771F881F991F1AF0BA9583
:1069E000C9F714C0B13091F00E94BA35B1E00895F2
:1069F0000C94BA35672F782F8827B85F39F0B93FE4
:106A0000CCF3869577956795B395D9F73EF4909535
:106A10008095709561957F4F8F4F9F4F0895E894B3
:106A200009C097FB3EF490958095709561957F4FD6
:106A30008F4F9F4F9923A9F0F92F96E9BB27939584
:106A4000F695879577956795B795F111F8CFFAF494
:106A5000BB0F11F460FF1BC06F5F7F4F8F4F9F4FC5
:106A600016C0882311F096E911C0772321F09EE823
:106A7000872F762F05C0662371F096E8862F70E089
:106A800060E02AF09A95660F771F881FDAF7880F63
:106A90009695879597F90895990F0008550FAA0BB9
:106AA000E0E8FEEF16161706E807F907C0F0121621
:106AB0001306E407F50798F0621B730B840B950B24
:106AC00039F40A2661F0232B242B252B21F4089579
:106AD0000A2609F4A140A6958FEF811D811D089516
:106AE00097F99F6780E870E060E008959FEF80EC81
:106AF000089500240A941616170618060906089524
:106B000000240A9412161306140605060895092E89
:106B10000394000C11F4882352F0BB0F40F4BF2BF8
:106B200011F460FF04C06F5F7F4F8F4F9F4F089538
:106B300057FD9058440F551F59F05F3F71F047952E
:106B4000880F97FB991F61F09F3F79F08795089513
:106B5000121613061406551FF2CF4695F1DF08C032
:106B6000161617061806991FF1CF8695710561054F
:106B700008940895E894BB2766277727CB0197F9F7
:106B800008950E944C3508F48FEF08950E94D9357E
:106B90000C9487350E94793538F00E94803520F0BA
:106BA000952311F00C9470350C94763511240C94C7
:106BB000BB350E94983570F3959FC1F3950F50E057
:106BC000551F629FF001729FBB27F00DB11D639F9F
:106BD000AA27F00DB11DAA1F649F6627B00DA11D45
:106BE000661F829F2227B00DA11D621F739FB00DEB
:106BF000A11D621F839FA00D611D221F749F33275B
:106C0000A00D611D231F849F600D211D822F762FF3
:106C10006A2F11249F5750409AF0F1F088234AF0D0
:106C2000EE0FFF1FBB1F661F771F881F915050403C
:106C3000A9F79E3F510580F00C9470350C94BB353C
:106C40005F3FE4F3983ED4F3869577956795B795C3
:106C5000F795E7959F5FC1F7FE2B880F911D9695DD
:106C6000879597F908950E944C35880B990B0895E4
:106C7000AA1BBB1B51E107C0AA1FBB1FA617B70762
:106C800010F0A61BB70B881F991F5A95A9F780957E
:106C90009095BC01CD010895A1E21A2EAA1BBB1B41
:106CA000FD010DC0AA1FBB1FEE1FFF1FA217B307D8
:106CB000E407F50720F0A21BB30BE40BF50B661FEE
:106CC000771F881F991F1A9469F7609570958095B2
:106CD00090959B01AC01BD01CF010895052E97FB56
:106CE0001EF400940E94853657FD07D00E944C3652
:106CF00007FC03D04EF40C948536509540953095A2
:106D000021953F4F4F4F5F4F089590958095709517
:106D100061957F4F8F4F9F4F0895EE0FFF1F059096
:106D2000F491E02D0994692796276927782787270A
:106D3000782708950E94A536A59F900DB49F900DC9
:106D4000A49F800D911D11240895A29FB001B39FAF
:106D5000C001A39F700D811D1124911DB29F700D64
:106D6000811D1124911D08950F931F93CF93DF93DD
:106D70008230910510F482E090E0E0910904F091F6
:106D80000A0430E020E0B0E0A0E0309799F421154B
:106D9000310509F44AC0281B390B24303105D8F5D8
:106DA0008A819B816115710589F1FB01938382833F
:106DB000FE0111C04081518102811381481759079A
:106DC000E0F04817590799F4109761F012960C9368
:106DD000129713961C933296CF01DF91CF911F919A
:106DE0000F9108950093090410930A04F4CF21151C
:106DF000310551F04217530738F0A901DB019A0120
:106E0000BD01DF01F801C1CFEF01F9CF90930A0472
:106E100080930904CDCFFE01E20FF31F819391937C
:106E20002250310939832883D7CF2091070430912C
:106E30000804232B41F42091020130910301309387
:106E400008042093070420910001309101012115CD
:106E5000310541F42DB73EB7409104015091050131
:106E6000241B350BE0910704F0910804E217F307A7
:106E7000A0F42E1B3F0B2817390778F0AC014E5FAA
:106E80005F4F2417350748F04E0F5F1F50930804DB
:106E900040930704819391939FCFF0E0E0E09CCF73
:106EA000CF93DF930097E9F0FC01329713821282AF
:106EB000A0910904B0910A04ED0130E020E01097A0
:106EC000A1F420813181820F931F2091070430911A
:106ED00008042817390709F061C0F0930804E0930B
:106EE0000704DF91CF910895EA01CE17DF07E8F597
:106EF0004A815B819E0141155105B1F7E901FB8390
:106F0000EA8349915991C40FD51FEC17FD0761F42D
:106F1000808191810296840F951FE901998388836E
:106F2000828193819B838A83F0E0E0E012968D91C9
:106F30009C9113970097B9F52D913C911197CD0134
:106F40000296820F931F209107043091080428179E
:106F5000390739F6309751F510920A041092090456
:106F6000B0930804A0930704BCCFD383C2834081AD
:106F70005181840F951FC817D90761F44E5F5F4F89
:106F800088819981480F591F518340838A819B8151
:106F9000938382832115310509F0B0CFF0930A0461
:106FA000E09309049ECFFD01DC01C0CF1382128261
:106FB000D7CF8F929F92AF92BF92CF92DF92EF92F4
:106FC000FF92CF93DF93EC01688179818A819B8165
:106FD000611571058105910521F464E279ED8BE578
:106FE00097E02DE133EF41E050E00E946E36490119
:106FF0005A019B01AC01A7EAB1E40E949A366B01E9
:107000007C01ACEEB4EFA50194010E944B3BC60E8F
:10701000D71EE81EF91EF7FE06C081E0C81AD10887
:10702000E10880E8F80AC882D982EA82FB82C701B7
:10703000B6019F77DF91CF91FF90EF90DF90CF90D7
:10704000BF90AF909F908F9008958F929F92AF9234
:10705000BF92CF92DF92EF92FF9260910601709102
:107060000701809108019091090161157105810561
:10707000910521F464E279ED8BE597E02DE133EFA2
:1070800041E050E00E946E3649015A019B01AC017B
:10709000A7EAB1E40E949A366B017C01ACEEB4EF32
:1070A000A50194010E944B3BC60ED71EE81EF91E97
:1070B000F7FE06C081E0C81AD108E10880E8F80AA6
:1070C000C0920601D0920701E0920801F0920901F6
:1070D000C701B6019F77FF90EF90DF90CF90BF90F0
:1070E000AF909F908F900895609306017093070171
:1070F00080930801909309010895FB01DC0104C00D
:107100008D910190801921F441505040C8F7881B9F
:10711000990B0895FB01DC0101900D920020E1F72D
:107120000895AEE0B0E0E7E9F8E30C945E3B0D892A
:107130001E8986E08C831A8309838FEF9FE79E83E5
:107140008D83AE01475E5F4F6F89788DCE010196CA
:107150000E94B4382F813885020F131FF801108266
:107160002E96E4E00C947A3BABE0B0E0EAEBF8E377
:107170000C94503B7C013B018A01FC011782168272
:10718000838181FFC8C1CE0101965C01F701938123
:10719000F30193FD859193FF81913F01882309F4C9
:1071A00053C1853239F493FD859193FF81913F015D
:1071B000853229F4B70190E00E94A43AE7CF912CE0
:1071C000212C312CFFE1F31538F08B3211F190F4C2
:1071D000803209F1833229F137FC3CC020ED280FC1
:1071E0002A3050F536FE20C08AE0989E200D1124EA
:1071F000922E06C08D3291F0803371F7689430F88A
:10720000F30193FD859193FF81913F018111DACFC5
:1072100021C0689431F8689432F8F2CF689433F85A
:10722000EFCF689434F8ECCFEAE02E9E200D1124C5
:10723000222E689435F8E4CF8E3229F436FC04C14E
:10724000689436F8DDCF8C3619F4689437F8D8CFC7
:107250008836B1F2982F9F7D95549330E0F08336B5
:10726000A1F18337C1F1833509F063C02801F2E051
:107270004F0E511CF801C080D180692D70E036FCA2
:1072800002C06FEF7FEFC6010E948E3A4C016894F6
:1072900037F882010AC00C5F1F4FFFE3F98388248F
:1072A0008394912C6501E89437F833FE2DC0522C5D
:1072B0008114910471F5552009F468CFB70180E27B
:1072C00090E00E94A43A5A94F6CFF8018081898315
:1072D0000E5F1F4FE4CF2801F2E04F0E511CF80162
:1072E000C080D180692D70E036FC02C06FEF7FEF67
:1072F000C6010E94993A4C018201D5CFB70180E2C4
:1073000090E00E94A43A2A942814190409F0B0F7D6
:10731000CECFF60137FC859137FE81916F01B70121
:1073200090E00E94A43A51105A94F1E08F1A91080B
:10733000BFCF843619F0893609F077C0F80137FEDF
:107340006BC060817181828193810C5F1F4FF32D2F
:10735000FF763F2E97FF09C09095809570956195B7
:107360007F4F8F4F9F4F689437F82AE030E0A50198
:107370000E94D43AC82ECA188C2C432C36FE0CC05E
:10738000E89440F8C91440F434FE05C032FC03C050
:10739000F32DFE7E4F2E892C44FE95C0FE01EC0D90
:1073A000F11D8081803309F087C0242D297E422E73
:1073B000842D8870582E43FC95C040FE8FC09C2CB5
:1073C000821418F42C0C922C981844FE91C0B7012A
:1073D00080E390E00E94A43A42FE09C088E790E072
:1073E00041FE02C088E590E0B7010E94A43AC914AA
:1073F00008F48AC0CA94D12C9FEFC91AD90ACA0CC2
:10740000DB1CF60182916F01B70190E00E94A43A63
:10741000AC14BD04B1F74FCF60817181072E000C11
:10742000880B990B0E5F1F4F92CFD32CE894D4F8A2
:107430002AE030E0853739F1232D297FD22E8F368F
:1074400001F148F48835A9F0F701868197812B96E0
:10745000E2E10C946C3B803749F08837A9F7D4FE01
:1074600002C06894D2F820E130E00DC06894D4F8EE
:10747000F6CF34FE03C0822F8660D82E20E132E0A2
:1074800002C028E030E0F801D7FE0FC060817181B2
:10749000828193810C5F1F4FA5010E94D43AC82EB0
:1074A000CA183D2CE89437F867CF6081718190E06D
:1074B00080E00E5F1F4FF0CF42FC02C0839478CF74
:1074C0008394839475CF842D867809F471CFF6CF99
:1074D000B70180E290E00E94A43A83948214C0F342
:1074E000512C73CF522C5818821408F46ECFF8CF59
:1074F000842D867809F47BCF8BE241FE80E247FC45
:107500008DE2B70190E071CFB70180E390E00E9477
:10751000A43A9A946CCF8FEF9FEF99CFFC0105901E
:10752000615070400110D8F7809590958E0F9F1F85
:107530000895FC016150704001900110D8F78095CA
:1075400090958E0F9F1F08950F931F93CF93DF93F6
:10755000182F092FEB018B8181FD09C01FEF0FEF61
:10756000812F902FDF91CF911F910F91089582FF6E
:1075700014C02E813F818C819D81281739073CF4EE
:10758000E881F981CF0101969983888310838E81E8
:107590009F8101969F838E83E3CFE885F985812FB4
:1075A0000995892BA1F3DACFFA01AA27283051F1E6
:1075B000203181F1E8946F936E7F6E5F7F4F8F4F24
:1075C0009F4FAF4FB1E03ED0B4E03CD0670F781F83
:1075D000891F9A1FA11D680F791F8A1F911DA11D68
:1075E0006A0F711D811D911DA11D20D009F46894A1
:1075F0003F912AE0269F11243019305D3193DEF649
:10760000CF010895462F4770405D4193B3E00FD0FE
:10761000C9F7F6CF462F4F70405D4A3318F0495DE9
:1076200031FD4052419302D0A9F7EACFB4E0A695CC
:107630009795879577956795BA95C9F700976105EE
:10764000710508959B01AC010A2E06945795479544
:1076500037952795BA95C9F7620F731F841F951F39
:10766000A01D0895F999FECF92BD81BDF89A992782
:1076700080B50895262FF999FECF1FBA92BD81BD1E
:1076800020BD0FB6F894FA9AF99A0FBE01960895A4
:10769000B7FF0C949A360E949A36821B930B08957A
:1076A0002F923F924F925F926F927F928F929F9212
:1076B000AF92BF92CF92DF92EF92FF920F931F9300
:1076C000CF93DF93CDB7DEB7CA1BDB0B0FB6F894B1
:1076D000DEBF0FBECDBF09942A88398848885F84F1
:1076E0006E847D848C849B84AA84B984C884DF8062
:1076F000EE80FD800C811B81AA81B981CE0FD11D46
:107700000FB6F894DEBF0FBECDBFED010895F8941B
:02771000FFCFA9
:1077120000000B04800001000000000425303258F4
:107722002530325825303258000057495A6E657458
:107732000000000000AF1F3620A21F9E2052205DD5
:10774200207B20D320D81F772038217821C51FCD58
:107752001FA51F00000000A7216A22A21FA621BDAB
:1077620021000000005E23A723A21F74235A23BB1B
:107772002304246F243D2386239B23B924A3231CA3
:1077820024E5233F2346235623000000007E2E31AA
:1077920030122E5E2EDE2DFA2DEC2D00000000C4DC
:1077A2002F0D0A006E616E00696E66006F766600CC
:00000001FF
